:108000000000012041150100BDEC0000BDEC0000A6
:10801000BDEC0000BDEC0000BDEC00000000000065
:10802000000000000000000000000000BDEC0000A7
:10803000BDEC000000000000BDEC00001D8600004B
:10804000BDEC0000BDEC0000BDEC0000BDEC00008C
:10805000BDEC0000BDEC0000BDEC0000BDEC00007C
:10806000BDEC0000BDEC0000BDEC0000BDEC00006C
:10807000BDEC0000BDEC0000BDEC0000BDEC00005C
:10808000BDEC0000BDEC0000BDEC0000BDEC00004C
:10809000BDEC0000BDEC0000BDEC0000BDEC00003C
:1080A000BDEC0000D1DB0000BDEC0000BDEC000029
:1080B000BDEC0000BDEC0000BDEC0000BDEC00001C
:1080C000BDEC0000BDEC0000BDEC0000BDEC00000C
:1080D000BDEC0000BDEC0000BDEC0000E5D70000E9
:1080E000BDEC0000BDEC0000BDEC0000BDEC0000EC
:1080F000BDEC0000BDEC0000BDEC0000BDEC0000DC
:10810000BDEC0000BDEC0000BDEC0000BDEC0000CB
:10811000BDEC0000D9FE0000BDEC0000BDEC00008D
:10812000BDEC0000BDEC0000BDEC0000BDEC0000AB
:10813000BDEC0000BDEC0000BDEC0000BDEC00009B
:10814000BDEC0000BDEC000071870000BDEC00003C
:10815000BDEC0000BDEC0000BDEC0000BDEC00007B
:10816000BDEC000021D80000BDEC0000BDEC00001B
:10817000BDEC0000BDEC0000BDEC0000BDEC00005B
:08818000BDEC0000BDEC0000A5
:10840000FFFFFFFFFFFFFFFFFFFFFFFF7EF9FFFF03
:1084100010B5054C237833B9044B13B10448AFF3BE
:1084200000800123237010BD0086FF1F00000000A4
:10843000241D01000C4B43B10C480D4910B5AFF39E
:1084400000800C48036823B910BD0A48036833B99B
:108450007047094B002BF7D0BDE810401847064B7A
:10846000002BF5D0184700BF00000000241D0100BC
:108470000486FF1F6C85FF1F0000000080F3118839
:1084800070472F4B41F238015A5842F478525A50F3
:108490002C4A927902F00C020C2A4FD041F244028D
:1084A0002949995003F558339A78110748BF9A78AB
:1084B000264944BF42F008029A70214B41F244021F
:1084C000995041F204015A5842F4803242F0C002FD
:1084D0005A501A6842F440221A6003F5E833242205
:1084E0005A701B4A80211170A2221A70DA7802F0A9
:1084F0001F02DA7003221A7100225A719A799207C8
:10850000FCD59A79D006FCD40E4B19469A7902F024
:108510000C02082AFAD140225A718B7903F00C031D
:10852000082BFAD1074B1A4699794906FCD5222126
:108530001970937903F00C030C2BFAD1704700BF2C
:1085400000700440004006400000330100001301A9
:10855000005006402B4B5A7902F0E0025A711A790A
:1085600002F0F8021A71284A136843F004031360FA
:10857000264A136823F0784323F001031360244B49
:108580001A7802F08C0242F050021A705A7802F007
:108590009C0242F040025A709A7802F0E6029A7009
:1085A0001C4A0023137083F311881B4B012283F8AC
:1085B000182383F81923022283F83C2383F83D23F0
:1085C00083F84B2383F84C2383F84D2383F84E2301
:1085D00083F84F23032283F81F2383F8212383F892
:1085E000232383F8252383F84223042283F82723B7
:1085F000052283F84923062283F83B23072283F8C8
:108600003523704700F007404080044000D0004010
:1086100000D0074000E0074000E100E00C4A13688A
:10862000013313600B4A1368013313600A4B1A6855
:108630003AB11A68013A1A601B6813B9074B012254
:108640001A70074B1A6812B11A68013A1A6070471B
:108650001C86FF1F6C080020B4030020B00300201C
:10866000B8030020024B034A5A6007221A60704781
:1086700010E000E000770100014B1868704700BF70
:108680001C86FF1F1449154B41F22802072888BF9A
:10869000002010B553F82030114CB4FBF3F48B5884
:1086A00043F480638B500F4B4FF440729A63422027
:1086B000DA6306F021FB0C4B0022DA709A709A7193
:1086C000DA725A71C4F30422E4B21A705C70DA7878
:1086D00042F02C02DA7010BD00700440E81A01006C
:1086E000C0C62D0000B0044000A00E40094A136827
:1086F00051680133202B08BF00238B4208D011683A
:10870000114408721360044AD37843F08003D37095
:10871000704700BF2086FF1F00A00E400A4B996AD9
:10872000DA6A91420DD09A6A511C1A44996292F801
:10873000302002709A6A202A01D100229A62012018
:1087400070470020704700BF2086FF1F044B1A7837
:1087500002F0FF0012B100221A700120704700BF22
:10876000B0030020014B1865704700BF2086FF1F33
:1087700030B526480179C9B28C0617D5244BDA6A80
:108780009C6A0132202A08BF0022A2421BBFDC6A79
:10879000C579C27918191EBFEDB280F83050DA627F
:1087A0001C4A052010601A6D1B4B1A604A0608D53A
:1087B0001A4B4FF480529A60144AD37803F0BF03E7
:1087C000D3700B061BD5144B1868C0B9104B196831
:1087D0005A68914214D0114A4FF4805151605A683E
:1087E000511C1A445960117A084AC9B2D1715968AA
:1087F000202908BF5860D37843F04003D37030BDC0
:10880000024AD37803F07F03F8E700BF00A00E40D0
:108810002086FF1FB4030020B803002080F00F4023
:1088200062B67047FFF7FCBF72B67047FFF7FCBF38
:108830004FF0E02318B1034AC3F80C2D7047024AE9
:10884000FAE700BF0400FA050100FA05F7B543484E
:10885000434C444D444E4FF480730E22436083607A
:10886000A2606261414A53629364D36413655365A5
:1088700093654FF4F0026A61AA603D4A4FF490712B
:1088800051621363936402F5342280324FF49051A5
:1088900091604FF48021516001F590515161354A4A
:1088A00040F20311116051609160D160116151611A
:1088B0009161D161304900224A6130490B614B61BD
:1088C0008B618B6601F5322101F580718E604E61FE
:1088D00003600826C360134611460A202A46B446A0
:1088E0001F46A646C4F804C00197019DB5F57A7FDE
:1088F0002AD3DEF81050A660ED0748BF013101977A
:10890000019DB5F57A7F23D3DEF81050ED0758BFEF
:1089100001330138E6D10A2919491DD10A2B1BD18F
:1089200001230B700D4B4FF4E0611960D96003F522
:1089300080534FF48071196001235360536943F0F1
:108940000103536103B0F0BD019D01350195CCE7F2
:10895000019D01350195D3E70023E2E70090044033
:1089600000F00F4040F00F407000000400A00440F1
:1089700000B0044000C00440C0F00F4000D00440EC
:10898000F3030020F7B5104B1B78D3B10F4B104DFC
:1089900002210F46042000241E469F605860019467
:1089A000019AAA4209D97160B0600194019AAA4261
:1089B000F3D8019A01320192F8E7019A013201924B
:1089C000EEE703B0F0BD00BFF303002000F00F405E
:1089D0001FA10700032806D8DFE800F00206080AF6
:1089E0001022054B5A6070472022FAE74022F8E730
:1089F0004FF08062F5E700BF00F10F40032806D872
:108A0000DFE800F00206080A1022054B9A60704762
:108A10002022FAE74022F8E74FF08062F5E700BF36
:108A200000F10F4010B50021044644FA01F3DB07C2
:108A3000C8B205D5FFF7CEFF01310829F5D110BD29
:108A4000FFF7DCFFF8E708B5032813D8DFE800F0EC
:108A5000020C0E10002004F049FF43F27C03984200
:108A600094BF0020012008BD0120F4E70220F2E7B6
:108A70000320F0E7002008BD032817D8DFE800F046
:108A800002070C110A4B1868C0F300107047084B1E
:108A90001868C0F340107047054B1868C0F3801089
:108AA0007047034B1868C0F3806070470020704720
:108AB00000F10F4070B5002425460126E0B2FFF713
:108AC000C2FF18B106FA04F31D43EDB20134082CBD
:108AD000F4D1284670BD024B1869C043C0B270473C
:108AE000C0F00F4008B5082004F000FF5E2811D93F
:108AF000134B1A780AB901221A70082004F0F6FE06
:108B000063280FD90F4B1B7863B90F4B4FF40072DA
:108B10005A6008BD082004F0E9FE5428EDD8002270
:108B2000074BE9E7082004F0E1FE542802D9054B81
:108B30001B781BB1044B4FF400729A6008BD00BF54
:108B40007486FF1FE403002080F00F40034B187869
:108B5000013801288CBF0020012070477486FF1F58
:108B6000034B1878012806BF02221A7000207047B4
:108B70007486FF1FC0B205F0F3BEC0B205F0DEBEC2
:108B80000B4B10F0010F4FF4800214BF5A609A6033
:108B900010F0020F4FF4001214BF5A609A6010F0E8
:108BA000040F4FF4801214BF5A609A60704700BFE0
:108BB00040F00F4008B507F0B3FF06F071FA06F079
:108BC00021FABDE8084008F02DB838B5054606F092
:108BD0006FF908280AD900242819013406F0E8F9A9
:108BE000092CF9D106F018FA012038BD002038BD53
:108BF000092106F07DB9002006F00ABC224923486D
:108C000041F23C028B5843F440538B50204B0121DE
:108C100019601A6802431A601E4ADA601A61DA6A39
:108C200042F08052DA621A6822F001021A601A6871
:108C300022F000621A60184A4FF400731360536008
:108C40009360D360136153619361D361A2F5F032F5
:108C500011601168014311601049D16001F52001D4
:108C60001161D16A41F08051D162116821F0010196
:108C70001160116821F00061116002F5E832936221
:108C8000D36213645364704700700440000C1F806B
:108C900000C002400300013E00B004400400513E09
:108CA000FF2810B54FEA004323D82B4C03F47C1364
:108CB0008AB141F000610B436363E36A002BFCDA85
:108CC000254BDA6AD000FCD5986BDA6A42F0104284
:108CD000C0B2DA6210BD41F000410B436363E36A46
:108CE000002BFCDAA06BE36A43F01043C0B2E362EE
:108CF00010BDB0F5007F17D2184C03F47C135AB1A5
:108D000041F000610B436363E36A002BFCDA134B11
:108D1000DA6AD100FCD5D7E741F000410B43636329
:108D2000E36A002BFCDADDE70D4C03F47C135AB147
:108D300041F000610B436363E36A002BFCDA084BEC
:108D4000DA6AD200FCD5BFE741F000410B43636310
:108D5000E36A002BFCDAC5E700C0024000D0024005
:108D600000C00A4010B5FFF787FC0446FFF784FCFB
:108D7000001B0028B8BF40420628F7DD10BD07B52C
:108D8000030A8DF805008DF80610032201A9A02022
:108D90008DF8043004F0B2FFFFF7E4FF03B05DF894
:108DA00004FBF0B5154600228BB00F461446AC42CA
:108DB00001D10BB0F0BD0AAB1344395D03F8221C9E
:108DC000531CC618F10602D0691E8C420DD1030A4D
:108DD0008DF80500033201A9A0208DF8043004F0BD
:108DE0008DFFFFF7BFFF3046002301341A46DEE750
:108DF0001FB5030A8DF80C30022203AB8DF80D006D
:108E000000921946A02004F0C5FF9DF80C0005B0A3
:108E10005DF804FB1FB5030A8DF80C308DF80D00CA
:108E200000920B46022203A9A02004F0B3FF05B074
:108E30005DF804FB30B4C0EBC000074C0D68255052
:108E400022188C8894808B79937100F5B0400722AA
:108E500030BCFFF7A6BF00BF7586FF1F054BC0EBF8
:108E6000C000184403680B6083888B8083798B7102
:108E7000704700BF7586FF1F30B500238BB001AD72
:108E80001A465A550133222BFBD14FF4B044230A22
:108E90008DF8054022222946A02020348DF8043088
:108EA00004F02CFFFFF75EFFB4F5484FEFD10B49FC
:108EB00000220C461346C2EBC20020440132B2F538
:108EC000805F0B704B708B70C37003714371837143
:108ED00001F10701EFD10BB030BD00BF7586FF1F58
:108EE00013B50C46C0EBC0000722694600F5B04040
:108EF000FFF790FF9DF8002023789A4212D19DF849
:108F0000012063789A420DD19DF80220A3789A42FD
:108F100008D1DDF80300D4F80330C31A5842584191
:108F200002B010BD0020FBE770477FB545F2FF702F
:108F3000FFF75EFF552802D12F4B1B78CBB30021E2
:108F400045F2FF70FFF71BFFFFF796FF40222B490A
:108F50002B4D0020FFF725FF4024204640222946C4
:108F60004034FFF71EFFB4F5E07FF6D104AD0023D7
:108F700045F8043D4FF4D36440F6780620460422B9
:108F800029460434FFF70DFFB442F7D100230393C1
:108F90004FF4FF6440F6D8062046042229460434E4
:108FA000FFF7FFFEB442F7D1552145F2FF70FFF7FE
:108FB000E6FE40221149134D0020FFF72BFF40240D
:108FC000A4F140012046402229444034FFF722FF0B
:108FD000B4F5E07FF4D158238DF8083000238DF8E4
:108FE00009304FF4E04300930222074B02A9A0206E
:108FF00004F0D0FE04B070BDF30300200C80FF1F0E
:10900000181B0100080400207586FF1F044B9B7885
:10901000052B044B8CBF042203221A70704700BF3B
:10902000580600207008002073B5D34D6A78A32A33
:109030002C4600F0848300F2E280132A00F09C8228
:1090400078D8072A00F0108238D8022A00F0AA81C6
:1090500008D8002A00F08581012A00F093810322BC
:1090600000F072BC052A00F0C68100F2DC81042AFF
:10907000F5D1D4F80300AD78C04E002856F825305D
:10908000B8BF4042984706EB8505A861A078202527
:1090900000F0010105FA01F1C9B2400804F04AFFED
:1090A000002840F0DF81A07806EB800600F0010187
:1090B00005FA01F141F00701B2696CE10F2A00F0F5
:1090C0002E8223D80D2A00F0EC8100F20C820C2AAB
:1090D000C5D1A878202500F0010105FA01F141F081
:1090E0001401C9B2400804F025FFA378D4F8032086
:1090F00003F0010105FA01F141F01401002A40F0EA
:10910000CD8140F00202C9B2580846E1112A9B4BBA
:1091100000F0248240F21582AD78D4F8030003EB0E
:1091200085031B6B984705F001032021994041F00E
:109130000A015CE11B2A00F0918236D8172A00F060
:109140003E8212D8152A00F032828C4B40F22282E5
:10915000AD78D4F8030053F82530984705F00103A3
:109160002021994041F0120141E1192A00F0518279
:1091700040F23382A878202500F0010105FA01F1C0
:1091800041F01401C9B2400804F0D4FEA378D4F829
:10919000032003F0010105FA01F141F01401002A56
:1091A00000F0598240F40062ADE7212A00F09C8271
:1091B00010D81F2A00F05B8200F275821C2A7FF40F
:1091C0004EAFD5F80310A878C9B202B0BDE8704020
:1091D00004F0CCBF8C2A00F09E82A22A00F0A68266
:1091E0007F2A7FF43CAFD5F80330022B00F2AB832B
:1091F000AA78624B1344EA7883F8482032E1B82A0F
:1092000000F0218351D8AB2A00F0DF8226D8A72AAC
:1092100000F0C08214D8A52A00F0A38240F2988200
:10922000A87805F0BFF8D5F80310AB78C9B20028CC
:1092300040F0AA82184602B0BDE8704004F006BFB4
:10924000A92A00F0B98240F2AE82D5F80310A878BE
:10925000C9B202B0BDE8704005F023B9B12A00F0F0
:10926000CF8210D8AD2A00F0C282C0F0B782AE2AF9
:109270007FF4F5AED5F80310A878C9B202B0BDE806
:10928000704005F03DB9B52A00F0C382B62A00F05F
:10929000CC82B32A7FF4E3AED5F80310A878C9B224
:1092A00002B0BDE8704004F0FBBFCA2A00F005839D
:1092B00031D8C12A00F0E28211D8BB2A00F0CC825A
:1092C000BC2A00F0D282B92A7FF4C9AED5F80310C7
:1092D000A878C9B202B0BDE8704004F0E7BEC32A66
:1092E00000F0DF82C0F0D282C92A7FF4B8AEA8783D
:1092F0001821400804F01EFE00F48062A878D5F81A
:10930000033000F00104202123F48063A14041F0E8
:1093100018011A433FE0D42A00F0EB8211D8D12A79
:1093200000F0D782D22A00F0DC82CC2A7FF497AEFC
:10933000D5F80310A878C9B202B0BDE8704005F0B6
:109340007DB9FB2A00F0DD82FF2A00F0F782D52AE2
:109350007FF485AEAA780A4B03EB8213EA785A763B
:1093600080E0A878202100F00103994041F00D0130
:10937000D5F803200FE000BF5806002078F6FF1F45
:1093800008040020A878D5F8032000F0010320216C
:10939000994041F00101C9B2400802B0BDE87040F7
:1093A00004F080BDA878D5F803302021002B00F010
:1093B000010301FA03F1C3BF0122C9B2D040C9B20F
:1093C000D8BF400804F06EFDAD78C34BD4F803005D
:1093D00001225A55C14B002853F82530B8BF4042EE
:1093E000984705F001032021994041F0070102460A
:1093F000C9B26808D1E7AC78B94BD5F803000022B0
:109400001A55B64B03EB84031B6B9847B54B43F8D7
:109410002400A878202100F00102914041F00601CB
:1094200053F82020B7E7A878202500F0010105FABD
:1094300001F141F01001C9B2400804F07BFDC3B254
:10944000A6780193E27806F0010105FA01F1D2084D
:1094500041F010010092C0F307430022C9B2700826
:1094600004F0C6FC02B070BDA878202400F0010111
:1094700004FA01F141F01001C9B2400804F05AFDAC
:10948000AE78EA7806F0010104FA01F1D208C0F3DF
:10949000072341F0100101920093DCE720F0020263
:1094A00031E6A878202100F00103994041F0140131
:1094B000C9B2400804F03EFDD5F803304BB9AB7893
:1094C000202103F00102914041F0140140F001021B
:1094D00019E6AB78202103F00102914041F014011C
:1094E00020F001020FE6A878202500F0010105FA1E
:1094F00001F141F01401C9B2400804F01BFDA3784A
:10950000D4F8032003F0010105FA01F141F0140140
:1095100012B140F01002F6E520F01002F3E5AC784D
:109520006E4BD5F8030003EB84031B6B984704F0E4
:1095300001032021994041F004010246C9B26008AC
:109540002BE7AD78D4F8030053F82530984705F0A1
:1095500001032021994041F0050148E7AC78D5F896
:10956000030003EB84031B6B984704F001032021E5
:10957000994041F00801E0E7AC78584BD5F803007A
:1095800053F82430984704F001032021994041F01A
:109590000301D2E7AD78D4F8030053F8253098479B
:1095A00005F001032021994041F00B011FE7A87845
:1095B000202100F00103994041F00C01D8E6AC787D
:1095C000464BD5F8030053F82430984704F00103C4
:1095D0002021994041F01301AFE7A878202500F041
:1095E000010105FA01F141F01401C9B2400804F08B
:1095F000A1FCA378D4F8032003F0010105FA01F1DE
:1096000041F0140112B140F008027CE520F008029C
:1096100079E5A878202100F00103994041F0140178
:10962000C9B2400804F086FCD5F803304BB1AB78E2
:10963000202103F00102914041F0140140F00402A6
:1096400061E5AB78202103F00102914041F0140163
:1096500020F0040257E520F4006254E5D5F8031029
:10966000A878C9B202B0BDE8704004F067BDA87820
:10967000202400F0010104FA01F141F01001C9B207
:10968000400804F057FCAE78EB7806F00101C2B256
:1096900004FA01F1C0F3072041F01001019200909B
:1096A00003F00F03D9E6A878010101F0100141F0A1
:1096B0006E01400804F03EFCAD78E3780193290187
:1096C000C0F3072001F01001002300901A4641F07A
:1096D0006E016808C4E600BFEB03002078F6FF1FA8
:1096E0005006002038060020A878010101F0100182
:1096F00041F06E01400804F01DFCAC78C0B201904E
:10970000EB780093210101F0100100231A4641F08B
:109710006E016008A4E6D5F80310A878C1F108012D
:10972000C9B202B0BDE8704004F0D8BCD5F803104F
:10973000A878C9B202B0BDE8704004F09FBCD5F86B
:109740000310A878C9B202B0BDE8704004F026BD8D
:10975000D5F80310A878C9B202B0BDE8704004F093
:109760004DBDA87804F01EFED5F80310C9B228B983
:10977000A87802B0BDE8704004F090BDA87802B0AF
:10978000BDE8704004F052BD184602B0BDE870401C
:1097900004F06CBDD5F80310A878C9B202B0BDE8DA
:1097A000704004F033BCD5F80310A878C9B202B0F9
:1097B000BDE8704004F0BABED5F80310A878C9B26D
:1097C00002B0BDE8704004F054BED5F80310A8788C
:1097D000C9B202B0BDE8704004F033BED5F8031042
:1097E000A878C9B202B0BDE8704004F072BED5F8E6
:1097F0000310A878C9B202B0BDE8704004F0AEBE54
:10980000D5F80310A878C9B202B0BDE8704004F0E2
:109810007DBCAC785E4BD5F8030053F824309847F4
:109820005C4B03EB841318611CE6AD78584BD4F8FD
:10983000030053F82530984705F001032021994093
:1098400041F01101D3E5D5F80310A878C9B202B0F0
:10985000BDE8704004F0BABCD5F80310A878C9B2CE
:1098600002B0BDE8704004F031BFD5F80310A8780D
:10987000C9B202B0BDE8704004F03EBFAA78454BC3
:1098800003EB8213D5F803201A72EBE5AD78404B59
:10989000D4F8030053F825309847AD013D4B58519B
:1098A000E0E5AC783A4BD5F8030053F824309847FC
:1098B000384B03EB84135860D4E5A878354BD5F8C2
:1098C000032003EB80135A8302B0BDE8704005F01B
:1098D00023B9D5F80310A87802B0BDE8704005F0B0
:1098E000E1B9A8782B4BD5F8032003EB8013DA619C
:1098F000EAE7AA78274B03EB8213D5F803201A6214
:10990000B0E5A8780021400804F014FBAB78D5F846
:10991000031013F0010F02464FEA530007D019B1AC
:1099200042F40072002138E522F4007235E511B1ED
:1099300042F48072F6E722F480722EE5D5F8032017
:109940002AB1012A12D00422134B1A708AE5A97891
:10995000104B03EB81131A760D4B104A43F821206C
:1099600003EB81031A651A639A667BE5A978094BB4
:1099700003EB81131A76064B094A43F8212003EBC7
:109980008103084A1A65084A1A63084AECE700BFCF
:1099900078F6FF1F0804002070080020E9EA0000A4
:1099A000F9E9000071EA000041EA0000B9EA0000AC
:1099B00038B5C14AC14C5378A42B154600F0CD826E
:1099C00000F2B880122B00F03D8257D8082B00F02F
:1099D000D88127D8032B00F09A8115D8012B00F0ED
:1099E0008E8140F271819078B54B03EB800320218A
:1099F0001D6D00F00103994041F00701C9B2400814
:109A000004F098FAA8476AE1052B00F09481C0F0B1
:109A10008A81062B00F09981072B00F0A581032392
:109A200023705DE10D2B00F0DF8111D80A2B00F0CF
:109A3000BA81C0F0B4810B2B00F0C7810C2BEED1A2
:109A40009078202100F00103994041F01401B1E128
:109A50000F2B00F0DF81C0F0CF81102B00F0E681EA
:109A6000112BDCD19078964B03EB800320219D6E67
:109A700000F00103994041F00801BFE71B2B00F003
:109A8000398228D8162B00F001820CD8142B00F054
:109A9000F18140F2E3819078202100F001039940A8
:109AA00041F00C0117E1182B00F00882C0F0FA8198
:109AB000192B00F011821A2BB1D19078202100F0DF
:109AC0000103994041F01401C9B2400804F032FA90
:109AD000C0F3C02003E1212B00F02A8214D81D2BF3
:109AE00000F01082C0F00A821F2B00F01382202B9E
:109AF00095D19078010101F0100141F06E0140080C
:109B000004F018FAC0B2EAE08C2B00F01C8207D8EF
:109B10007F2B84D192786A4B134493F8483052E1FA
:109B2000A22B00F01682A32B7FF479AF907804F07B
:109B300039FCD4E0BC2B00F065825DD8AD2B00F081
:109B400039821BD8A82B00F0258208D8A62B00F05C
:109B5000158240F20682907804F0BAFBBFE0AA2B8F
:109B600000F02082C0F01A82AB2B00F01F82AC2BD9
:109B70007FF455AF907804F02DFDB0E0B52B00F0E8
:109B80002F821CD8B12B00F0198206D8AE2B7FF49F
:109B900046AF907804F02AFDA1E0B32B00F01C82C0
:109BA000B42B7FF43CAF9078010101F0100141F03B
:109BB0006F01400804F0BEF9C0F304408FE0B82BF9
:109BC00000F018820ED8B62B7FF429AF90783C4B6A
:109BD00003EB800320211D6D00F00103994041F04B
:109BE00011010BE7B92B00F00982BB2B7FF417AFF3
:109BF000907804F0BBFD72E0CC2B00F0308220D8CE
:109C0000C32B00F012820BD8C12B00F0FF8100F2B1
:109C10000382BD2B7FF403AF907804F0BEFD5EE0BD
:109C2000C52B00F01182C0F00A82C92B00F00F8210
:109C3000CA2B7FF4F4AE9278224B03EB82135B8B3A
:109C4000C1E0D22B00F02E821CD8CF2B00F00B826B
:109C50000ED8CE2B7FF4E3AE9078010101F0100115
:109C600041F06F01400804F065F9C0F3090036E0E7
:109C7000D02B00F00C82D12B7FF4D1AE907805F080
:109C800007F82CE0D52B00F0138208D8D42B7FF4F2
:109C9000C6AE92780B4B03EB82131B6A93E0FB2B4F
:109CA00000F00C82FF2B7FF4BAAE9278054B03EBE9
:109CB00082131B7E87E000BF58060020700800203A
:109CC00078F6FF1F080400209078202100F001039F
:109CD000994041F00D01C9B2400804F02BF96060D1
:109CE000B84B1B7853B1B84B62681A60B74B002A67
:109CF00040F0F1811A6842F008021A6038BD90788D
:109D0000202100F00103994041F00101E3E7907840
:109D1000AF4B03EB800320211D6D00F00103994040
:109D200041F002016AE69278A94B03EB82031A6DB7
:109D300098699047D3E79278A54BA64903EB820335
:109D400051F822009B6E9847C9E79078202100F0D7
:109D50000103994041F01001C9B2400804F0EAF84B
:109D6000C0F30720C000BAE79078202100F001037B
:109D7000994041F01001C9B2400804F0DBF8C0B2CC
:109D8000F0E79078202100F00103994041F015019F
:109D9000C9B2400804F0CEF8C0F340209FE79078A5
:109DA00004F018FE9BE79078202100F00103994011
:109DB00041F01501C9B2400804F0BCF810F0020FE0
:109DC0000CBF0123002363608AE79078202100F014
:109DD0000103994041F01501C9B2400804F0AAF806
:109DE000C04300F001007AE79078202100F00103E1
:109DF000994041F01401EFE79078202100F0010331
:109E0000994041F01401C9B2400804F093F8C0F33E
:109E1000001064E790786E4B03EB800320219D6E69
:109E200000F00103994041F00401E7E59078684BA8
:109E300003EB800320211D6D00F00103994041F0E8
:109E40000501DBE59078624B03EB800320219D6EDA
:109E500000F00103994041F00A01CFE590785C4B96
:109E600003EB800320211D6D00F00103994041F0B8
:109E70000301C3E59078564B03EB800320211D6D51
:109E800000F00103994041F00B01B7E59078504B89
:109E900003EB800320211D6D00F00103994041F088
:109EA0001201ABE590784A4B03EB800320211D6D36
:109EB00000F00103994041F013019FE590782021C3
:109EC00000F00103994041F01401C9B2400804F0C8
:109ED00031F8C0F3C00002E79078202100F00103C0
:109EE000994041F01401C9B2400804F023F8C0F3CE
:109EF0008000F4E6907804F03DFAF0E6907804F003
:109F000045FAECE69078324B03EB80031D6D02F0CE
:109F1000CBFC77E59078202100F00103994041F0D7
:109F20001001C9B2400804F005F8C0F30340D6E6BA
:109F30009078010101F0100141F06E01400803F03A
:109F4000F9FF0012CBE6907804F0FCF9C0F10800AC
:109F5000C5E6907804F0DEF9C1E6907804F03AFAAC
:109F6000BDE6907804F01EFAAB7818B9184604F0F4
:109F70005AFAB4E6184604F039FAB0E6907804F0DC
:109F800011FA18B9A87804F0B9F9A8E6A87804F08D
:109F90003EFAA4E6907804F039FBA0E6907804F04D
:109FA00001FB9CE6907804F009FB98E6907804F0B9
:109FB000EDFA94E6907804F035FB90E6907804F0A2
:109FC000CDF98CE66B0800205C08002060060020BC
:109FD00078F6FF1F38060020907804F026FA7EE617
:109FE00091783F4B3F4A03EB811302EB81021869E2
:109FF000126D9EE6907804F0E1F970E6907804F036
:10A0000095F96CE6907804F0BDFB68E69278344BE5
:10A0100003EB82131B7AD6E69278324B910103EB65
:10A0200082032F4A1B6D50588DE691782C4B2D4A98
:10A0300003EB811302EB81025868126D79E6927886
:10A04000294B53F82230BEE69278284BF9E79078F6
:10A05000202100F00103994041F018013BE690787F
:10A0600004F060FB3BE6002363609378204AD15CF8
:10A0700009B1012161600021D1541E4AD15C19B19E
:10A08000616841F0020161600021D15428E69078B6
:10A09000010101F0100141F06F01400803F04AFF97
:10A0A00000161CE692780E4B03EB8213DB698AE6FE
:10A0B00092780B4B03EB82135B7E84E6907810F072
:10A0C00001014FEA500001D0002163E603F032FFA6
:10A0D000C0F3002003E61A6822F008020DE600BF74
:10A0E0000804002078F6FF1FC40300208C05002020
:10A0F00000040020E503002038B5C24A9378022B03
:10A10000144600F00881032B00F00C81002B40F076
:10A11000378253784E2B00F0B48030D8462B00F0B5
:10A12000828012D8422B6ED006D8402B5FD0412BB4
:10A1300064D00322B44B58E0442B69D0452BF8D1AE
:10A14000B24BD1785971052054E04B2B00F0898037
:10A150000BD8472B6FD0492BEBD1D278AB4B002AD1
:10A160007AD1DA75D97D172044E04C2B00F0848039
:10A170004D2BDED1A54BD178597515203AE0542BE3
:10A1800000F0A6801BD8512B00F08D8009D84F2BF2
:10A1900000F08280502BCCD19C4BD1789975162041
:10A1A00028E0522B00F08C80532BC2D1974DD2F86F
:10A1B00003302946042241F8103F102043E0842B4D
:10A1C00000F09E800AD8552B00F08E80832BB0D1F2
:10A1D0008F4BD2F80320C3F8802038BD852B00F0C8
:10A1E0009480FF2BA5D1D2788A4B1A7038BDD178D4
:10A1F00045F2FF70BDE83840FEF7C1BD834BD17812
:10A2000019700020F6E7814BD17859700120F1E7F1
:10A210007E49D2F8033041F81C3F04221C20BDE8DF
:10A220003840FEF7BEBD7949D2F8033041F80C3F03
:10A2300004220C20F3E7754DD2F80330294604229E
:10A2400041F8083F0820FEF7ACFD2A8A2989687981
:10A25000BDE8384003F07ABB6B490122DA754A60E9
:10A2600080E76A4CD178E1700320FEF788FDE07842
:10A27000BDE83840FEF776BA644BD1789970022079
:10A28000B8E7624CD2F80300E084FEF779FC0222C2
:10A2900004F126012620C2E7D2F803105B4BC9B2B5
:10A2A00059761920A6E7594D2A7DD20704D5E378BF
:10A2B000DB0701D4FEF7E0FDE1782975142099E76A
:10A2C0005249D2F8033041F8203F04222020A6E76B
:10A2D000D2F80330012B00F253814C49D37801F8B6
:10A2E0001A3F01221A209AE7D2F80330012B00F21C
:10A2F00047814649D37801F81B3F01221B208EE796
:10A30000454BD2F803201A6038BD414BD2F80320E8
:10A31000C3F8842038BD5178404BD2F8032043F86D
:10A32000212038BD53782E2B3FF603AF01A252F8FF
:10A3300023F000BFF1A3000025A4000039A4000011
:10A3400033A1000033A1000033A1000033A10000BD
:10A3500033A1000033A100004DA4000057A4000069
:10A3600061A400006BA4000075A400007FA400009D
:10A3700033A1000033A1000033A1000033A100008D
:10A3800033A1000033A1000033A1000033A100007D
:10A3900033A1000033A1000033A1000033A100006D
:10A3A00089A4000097A40000A5A40000B3A40000A5
:10A3B000C1A40000CFA40000DDA40000EBA40000B5
:10A3C000F9A4000007A5000015A5000023A50000C2
:10A3D00031A500003BA5000045A500004FA50000E9
:10A3E00059A5000063A500006DA5000077A5000039
:10A3F0000B4BD4F803201A60FEF73EF9044BC3F868
:10A40000880038BD58060020700800200C80FF1F0F
:10A4100078F6FF1F6A0800206C0800207C080020E6
:10A42000A4050020574BD4F803205A60FEF724F906
:10A43000554BC3F88C0038BD524BD4F803209A60BA
:10A44000FEF71AF9504BC3F8900038BD4D4BD4F8C5
:10A450000320DA6038BD4B4BD4F803201A6138BDB5
:10A46000484BD4F803205A6138BD464BD4F803203A
:10A470009A6138BD434BD4F80320DA6138BD414BB3
:10A48000D4F803201A6238BDD4F803303D4ADBB259
:10A4900082F8243038BDD4F803303A4ADBB282F86F
:10A4A0002A3038BDD4F80330364ADBB282F8253082
:10A4B00038BDD4F80330334ADBB282F82B3038BDD4
:10A4C000D4F803302F4ADBB282F8263038BDD4F8F6
:10A4D00003302C4ADBB282F82C3038BDD4F803307C
:10A4E000284ADBB282F8273038BDD4F80330254A39
:10A4F000DBB282F82D3038BDD4F80330214ADBB20C
:10A5000082F8283038BDD4F803301E4ADBB282F816
:10A510002E3038BDD4F803301A4ADBB282F8293025
:10A5200038BDD4F80330174ADBB282F82F3038BD7B
:10A53000144BD4F803201A6338BD124BD4F803200F
:10A540005A6338BD0F4BD4F803209A6338BD0D4BC6
:10A55000D4F80320DA6338BD0A4BD4F803201A6418
:10A5600038BD084BD4F803205A6438BD054BD4F8E5
:10A5700003209A6438BD034BD4F80320DA6438BD55
:10A580000422D7E5A405002078F6FF1F2DE9F04F3F
:10A59000C74EC84F32787A7064233B70212AD6F8B0
:10A5A00003307B6087B035463C4601F0BB8100F24A
:10A5B000C7800E2A00F0558639D8072A00F0578444
:10A5C00014D8032A00F06E8208D8012A00F09F8177
:10A5D000022A00F0048202232370FAE1052A00F027
:10A5E000438440F29F82FFF7E3F9F2E10A2A00F088
:10A5F000448407D8082A00F03D84092AEBD1FFF7EC
:10A600007BFDE6E10C2A00F0F98540F2CB85B078BD
:10A61000052800F2E1817378012B00F00786C0F075
:10A620000186022B00F0068603233B70D1E1182A35
:10A6300000F0638730D8142A00F09D8615D80F2AC1
:10A6400000F02E86132AC6D171789B4A092900F2A0
:10A650006686DFE811F061066D0670067306770600
:10A660007E068106840687067C06162A00F040874F
:10A6700040F2A286914AD2F89C10072900F2A981E3
:10A68000481C02EB8101C2F89C00D2F89800C1F886
:10A69000A000C2F898309CE11C2A01F04B8022D81F
:10A6A0001A2A00F04C8740F23987844C94F8C12074
:10A6B00072B95E1C04BF804B1B680A205843C4F863
:10A6C000C400FDF7D9FF0123C4F8C80084F8C130E5
:10A6D0006B78042B00F27D81DFE813F042078707D7
:10A6E000BE07F5075A071F2A01F0628001F2B38006
:10A6F0001E2A7FF470AF7278142A00F26285B67851
:10A70000052E01F21D8006206D4C00FB026144F80D
:10A7100021306C4B9B7E002B00F05B81002A00F007
:10A72000588110FB02611820013A424302F5D360C0
:10A73000042204EB810102FB0600FEF732FB48E134
:10A74000802A01F0DA8144D8402A01F0BE8129D85C
:10A75000242A01F045810CD8222A01F03981232ACC
:10A760007FF439AF544B1B68C6F80330FFF7C4FCC5
:10A770002FE1262A01F08081C1F06581272A7FF42C
:10A780002AAFB278052A00F227817378142B00F2E1
:10A790001885062101FB0323474A1168484A42F8FD
:10A7A000231016E1442A01F09C8107D8422A01F0C7
:10A7B000948141F28E8102F070F80AE1462A01F09C
:10A7C0009881C1F09281472A7FF405AF02F069F8C1
:10A7D000FFE0872A01F02D8246D8832A01F0AC8160
:10A7E0000AD8812A01F08F81822A7FF4F4AE334B9C
:10A7F000022283F89420ECE0852A01F0D281314ACC
:10A8000041F2BC813049314C01250D70B3F5805FB8
:10A810009178217081F0CB81127D12EA050641F01A
:10A82000C681184604A9FEF719FB9DF81030637025
:10A830009DF81130A3709DF81230E3709DF816302A
:10A8400023719DF8153063719DF81430A3719DF844
:10A850001330E37126722B46E15C227A01330A44FD
:10A86000082B2272F8D1B4E08C2A01F02B823BD85D
:10A87000892A01F00C82C1F0A4818A2A7FF4ABAE50
:10A880007278134B002A41F01A821A70114AEB7841
:10A8900013700A4A92F8B0110F4A11700F49002242
:10A8A0000A700F490A700F4A11780B43137090E039
:10A8B00058060020700800205C08002078F6FF1F72
:10A8C000640600200C80FF1F600800206108002043
:10A8D000DC030020F203002007060020F103002023
:10A8E00056060020DD030020F22A01F07182FF2AC3
:10A8F00001F0B3828D2A7FF46EAE7278032A01F2E2
:10A900006382DFE812F01F0A060A380A460AB378A3
:10A91000052B61D8DFF8F8B2DFF8F8820024AA78B6
:10A92000E6B2B2420AD0B44B03EB8212527E002A46
:10A930004CD003EB84135B7E934247D1AF4B14F8AA
:10A9400008204FF0000906F0010704F8039004F80E
:10A950000B904FEA840A760862B12021B940A84AD8
:10A9600041F0060152F82420C9B2304603F09AFAA9
:10A9700004F80890A34AD5F803004FF0010904F841
:10A980000290A14A002852F80A304FF02001B8BFC7
:10A99000404201FA07F79847F6B247F0070102462E
:10A9A000C9B2304603F07EFAD5F80330002BD8BF89
:10A9B00002224FF00003D8BF0192F9B2C8BFCDF810
:10A9C000049000931A46304603F012FA0134062C24
:10A9D000A5D107B0BDE8F08F04232370F9E7B37861
:10A9E000052BF9D8DFF828B2DFF828820024AA78EE
:10A9F000E6B2B2420AD0804B03EB8212527E002AAA
:10AA00004CD003EB84135B7E934247D17B4B14F80D
:10AA100008204FF0000906F0010704F8039004F83D
:10AA20000B904FEA840A760862B12021B940744A3B
:10AA300041F0060152F82420C9B2304603F032FA40
:10AA400004F808906F4AD5F803004FF0010904F8A4
:10AA500002906D4A002852F80A304FF02001B8BF2A
:10AA6000404201FA07F79847F6B247F0070102465D
:10AA7000C9B2304603F016FAD5F80330002BC8BF30
:10AA800002224FF00003C8BF0192F9B2D8BFCDF83F
:10AA9000049000931A46304603F0AAF90134062CBC
:10AAA000A5D196E7B378052B96D8DFF85881DFF863
:10AAB0004C91DFF85CA10026AA78F4B2A24209D03A
:10AAC0004D4B03EB8212527E42B303EB86135B7E47
:10AAD000934223D1204602F077FE012304EA0300CB
:10AAE0004FF0200B0BFA00FB24FA03F74BF00701A1
:10AAF00006F808300022C9B2384603F0D3F9002422
:10AB0000022301930094234622465FFA8BF13846D4
:10AB100003F06EF906F8094006F80A400136062EE1
:10AB2000CAD156E7B078052803D97278022A7FF493
:10AB300050AF6A78012A6FD005D3022A00F0E9806D
:10AB40000323237045E7DFF8B490DFF8C4A0DFF8F3
:10AB5000B4800024AA78A2420AD0274B03EB8212C9
:10AB6000527E002A44D003EB84135B7E93423FD194
:10AB700014F808304FF0000B04F809B004F80AB0DC
:10AB800004F00107660863B12021204BB94041F071
:10AB9000070153F82420C9B2F0B203F083F904F896
:10ABA00008B0DFF870B014F80B306BB12021144BF3
:10ABB000B94041F0060153F82420C9B2F0B203F0C5
:10ABC00071F9002304F80B30202303FA07F7F6B2DB
:10ABD00047F00D01D5F80320C9B2304603F062F901
:10ABE0000023019300931A46F9B2304603F000F9AE
:10ABF0000134062CAED1ECE608040020E503002069
:10AC000038060020EB03002078F6FF1F90F6FF1FA8
:10AC10000004002050060020DFF800A3DFF808B38E
:10AC20000026AA78B2420AD0B54B03EB8212527EBC
:10AC3000002A57D003EB86135B7E934252D1B14B6F
:10AC40004FF0000806F8038016F80B3006F80A806B
:10AC5000012B4FF0200106F001094FEA56074FD0B3
:10AC600044D3022B51D0A84BF25C7AB1202101FAD7
:10AC700009F1A64A039341F0070152F82620C9B210
:10AC8000F8B203F00FF9039B0022F254A04BF25CE0
:10AC90007AB1202101FA09F19E4A039341F006019D
:10ACA00052F82620C9B2F8B203F0FCF8039B002248
:10ACB000F254D5F803309844202303FA09F9FFB27F
:10ACC00049F00D014246C9B2384603F0EBF80023C3
:10ACD000019300931A465FFA89F1384603F088F829
:10ACE000C4F804800136062E9BD172E601FA09F100
:10ACF00041F00D01C9B2F8B203F01CF98046B2E789
:10AD000001FA09F141F00101F4E7F0B203F0C0FFEC
:10AD1000F4E7142B3FF760AE030654D5DFF8E49157
:10AD2000DFF8F8A1DFF8E0810024AB782341DF07EA
:10AD300045D514F808304FF0000B04F809B004F8BA
:10AD40000AB004F00107660863B120216F4BB940D7
:10AD500041F0070153F82420C9B2F0B203F0A2F881
:10AD600004F808B0DFF8A8B114F80B306BB120215B
:10AD7000684BB94041F0060153F82420C9B2F0B243
:10AD800003F090F8002304F80B30202303FA07F7B0
:10AD9000D5F80330062202FB03435F4AF6B247F0C0
:10ADA0000D0152F82320C9B2304603F07BF800238E
:10ADB000019300931A46F9B2304603F019F80134B2
:10ADC000062CB2D105E605283FF606AE4D4B4E4E99
:10ADD00000241C54514B1C54335C7BB1504B00F08D
:10ADE0000102202103EB8003914041F007019A69A1
:10ADF000C9B2400803F056F8AB78F454A878444C34
:10AE0000235C7BB100F0010320219940414B41F0CC
:10AE1000060153F82020C9B2400803F043F8AB788C
:10AE20000022E254A878D5F803302024062200F04E
:10AE3000010102FB030304FA01F1374A41F00D015D
:10AE400052F82320C9B2400803F02CF8A87800F08B
:10AE50000101002304FA01F1019300931A46C9B2DB
:10AE6000400802F0C5FFB4E5FEF7DEF8B1E5FEF7F5
:10AE7000CDF8AEE5FEF7CAF8ABE5B378022B00F0EB
:10AE8000D280032B00F0D480002B40F084817378B3
:10AE9000502B00F09A8025D8472B00F0868011D8DF
:10AEA000422B79D006D8402B5CD0412B70D00323A5
:10AEB00023705CE0452B72D074D8442BF7D1194B2A
:10AEC000DB6967E04C2B79D006D8492B70D04B2B2F
:10AED000EDD1144BDB785DE04E2B124B73D070D963
:10AEE0005B7E57E0802B7FD029D8532B73D01DD8A1
:10AEF000512B6DD0522BDAD10A4B1B6A4AE000BFAE
:10AF000008040020E5030020EB03002090F6FF1F5B
:10AF100050060020380600206406002000040020AF
:10AF200078F6FF1F0C80FF1FC0F6FF1F552B58D06F
:10AF300054D3562BBBD1A64B93F824302AE0832B55
:10AF40005DD007D8812B53D0822BB0D1A14BD3F841
:10AF500098301FE0852B59D055D3FF2BA7D19E4B9E
:10AF60001B7827E045F2FF70FDF742FF78609B4BAE
:10AF70001B78002B3FF42DAD994B62681A60994BFA
:10AF8000002A40F00A811A6842F008021A6020E59F
:10AF90008F4B1B786360EAE78D4B5B78FAE78C4B4D
:10AFA0005B79F7E78A4BDB68F4E7894B9B68F1E74D
:10AFB000874BDB7D003318BF0123EBE7844B9B7885
:10AFC000E8E75B7DE6E7DB8CE4E7814B9B7DE1E72F
:10AFD0007F4B1B7DDEE77E4B1B69DBE77C4B9B7E5B
:10AFE000D8E77B4BDB7ED5E77A4B93F89430D1E7FB
:10AFF000784B93F894301E1F73427341CAE7754B28
:10B00000D3F88030C6E7784B1B68C3E7714A7748AE
:10B01000D2F8843043F2390100FB0313C2F88430C4
:10B0200023F00043B6E77278714B53F82230B1E752
:10B0300073782E2B3FF63BAF01A252F823F000BFEE
:10B04000FDB0000001B1000007B10000AFAE00008C
:10B05000AFAE0000AFAE0000AFAE0000AFAE00007C
:10B06000AFAE00006FAF00006FAF00006FAF000029
:10B070006FAF00006FAF00006FAF0000AFAE000019
:10B08000AFAE0000AFAE0000AFAE0000AFAE00004C
:10B09000AFAE0000AFAE0000AFAE0000AFAE00003C
:10B0A000AFAE0000AFAE0000AFAE00000BB10000CD
:10B0B0000FB1000017B100001FB1000027B1000060
:10B0C0002FB1000037B100003FB1000047B10000D0
:10B0D0004FB1000057B100005FB1000067B1000040
:10B0E0006DB1000073B1000079B100007FB10000C4
:10B0F00085B100008BB1000091B100003D4B83E7AA
:10B100003C4B5B6846E73B4B50E73A4B14E7394B07
:10B1100093F82A303EE7374B93F825303AE7354B22
:10B1200093F82B3036E7334B93F8263032E7314B28
:10B1300093F82C302EE72F4B93F827302AE72D4B2E
:10B1400093F82D3026E72B4B93F8283022E7294B34
:10B1500093F82E301EE7274B93F829301AE7254B3A
:10B1600093F82F3016E7234B1B6B13E7214B5B6BD8
:10B1700010E7204B9B6B0DE71E4BDB6B0AE71D4B6B
:10B180001B6C07E71B4B5B6C04E71A4B9B6C01E7DE
:10B19000184BDB6CFEE604238AE61A6822F00802EC
:10B1A0001A6016E4B378022B0ED17078372808D8CD
:10B1B00000F5FF701049800004220144FDF7F1FD05
:10B1C00007E40323237004E404233B7001E400BF7D
:10B1D0000C80FF1F78F6FF1F6A0800206B08002014
:10B1E0005C080020600600206C0800206D4EC641FF
:10B1F0007C080020A405002084000020B378022BE6
:10B200000CD170783728DCD800F5FF70A349800096
:10B2100004220144FDF7FEFDFFF7DBBB04233B7076
:10B22000FFF7D7BB02F0C8FAFFF7D3BB02F0CCFAA6
:10B23000FFF7CFBB02F0D0FA994B78601B78002B58
:10B240003FF4C7AB974B1860974B1A6820B942F090
:10B2500008021A60FFF7BDBB22F008021A60FFF770
:10B26000B8BBB278022A17D17078072808D81BB962
:10B27000FDF7C4FBFFF7ADBBFDF7ACFBFFF7A9BBC8
:10B28000FF287FF4A6AB5D1C0ABF864BD8B21878A6
:10B29000FDF7C8FBFFF79DBB04233B70FFF799BB8D
:10B2A000B378012B2AD023B1022B2BD004233B707F
:10B2B0000FE07078082803D8FDF7C5FB606008E050
:10B2C0000A2816D1794B1B6983F40073C3F340231A
:10B2D0007B60734B1B78002B3FF47BAB714B626838
:10B2E0001A60714B92B91A6842F008021A60FFF7AF
:10B2F00070BBFF28EDD1FDF7DDFBDFE7707802F0D2
:10B30000F5FADBE77078FDF7B7FBD7E71A6822F0AC
:10B3100008021A60FFF75DBB1068184410601268DD
:10B32000614B12BB1A6842F008021A60FFF751BB6A
:10B330001068C01AF2E710685843EFE7106890FBF6
:10B34000F3F0EBE7116891FBF3F003FB10131360CC
:10B35000E5E710681840E1E710681843DEE7106879
:10B360005840DBE71368DB43F1E71A6822F0080274
:10B370001A60FFF72EBB4B4A11684B4A8B42136889
:10B380000BDA23F0030343F004031360136871B96D
:10B3900043F008031360FFF71CBB0BBF23F0060349
:10B3A00023F0050343F0010343F00203EDE723F02C
:10B3B00008031360FFF70DBB72780C2A3FF609AB48
:10B3C000DFE802F007111B252F39444E58627882BE
:10B3D0008C00354A126814077FF5FBAA344AC2F87C
:10B3E0009830FFF7F6BA304A126810073FF5F1AA15
:10B3F0002F4AC2F89830FFF7ECBA2B4A1268D107EF
:10B400007FF5E7AA2A4AC2F89830FFF7E2BA264A3F
:10B410001268D2073FF5DDAA254AC2F89830FFF737
:10B42000D8BA214A126857077FF5D3AA204AC2F832
:10B430009830FFF7CEBA1C4A126812F0050F3FF49D
:10B44000C8AA1B4AC2F89830FFF7C3BA164A126856
:10B4500096077FF5BEAA164AC2F89830FFF7B9BA28
:10B46000114A126895073FF4B4AA114AC2F89830FD
:10B47000FFF7AFBA0C4A1268D4067FF5AAAA0C4AA5
:10B48000C2F89830FFF7A5BA074A126890067FF510
:10B49000A0AA074AC2F89830FFF79BBA84000020A0
:10B4A0006B0800205C0800206006002080F00F4040
:10B4B00078F6FF1FBA4A126851067FF58AAAB94A80
:10B4C000C2F89830FFF785BAB54A126812067FF5C0
:10B4D00080AAB44AC2F89830FFF77BBAB04A126823
:10B4E000D7057FF576AAAF4AC2F89830FFF771BA50
:10B4F000AC4AC2F89830FFF76CBAAA4AD2F89C302E
:10B50000002B3FF466AA013BC2F89C3002EB830398
:10B51000D3F8A030C2F89830FFF75BBA73782E2BBF
:10B5200004D8A14A0121D154FFF753BAFF2B7FF46D
:10B5300048AE9C4B012283F8C020FFF74ABA7378CB
:10B540002E2B04D8984A0021D154FFF742BAFF2B82
:10B550007FF437AE934B002283F8C020FFF739BA4F
:10B56000FDF78AF8D4F8C830C01A0028D4F8C430DF
:10B57000B8BF4042984295BFD4F89830002303F1F9
:10B58000FF3384F8C13098BFC4F89830FFF721BA70
:10B59000A87802F021F940B9814A84F8C100136803
:10B5A00023F010031360FFF714BAD4F8C430ABB122
:10B5B000FDF762F8D4F8C830C01A0028D4F8C430B7
:10B5C000B8BF4042984209D9754A002384F8C13077
:10B5D000136843F010031360FFF7FBB9D4F89830F9
:10B5E000013BC4F89830FFF7F4B9A878202100F0A7
:10B5F0000103994041F01501C9B2400802F09AFCDC
:10B6000010F4007509D0664A002384F8C13013682D
:10B6100023F010031360FFF7DCB9D4F8C430A3B1F2
:10B62000FDF72AF8D4F8C830C01A0028D4F8C4307E
:10B63000B8BF4042984208D9594A84F8C1501368AB
:10B6400043F010031360FFF7C4B9D4F89830013BFE
:10B65000C4F89830FFF7BDB9A878202100F00103A5
:10B66000994041F01501C9B2400802F063FC10F0A6
:10B67000010509D04A4A002384F8C130136823F039
:10B6800010031360FFF7A5B9D4F8C430A3B1FCF7D9
:10B69000F3FFD4F8C830C01A0028D4F8C430B8BFBB
:10B6A0004042984208D93E4A84F8C150136843F09A
:10B6B00010031360FFF78DB9D4F89830013BC4F83C
:10B6C0009830FFF786B9A878202100F0010399404F
:10B6D00041F01501C9B2400802F02CFC10F002053F
:10B6E00009D02F4A002384F8C130136823F01003D7
:10B6F0001360FFF76EB9D4F8C430A3B1FCF7BCFFF8
:10B70000D4F8C830C01A0028D4F8C430B8BF4042BA
:10B71000984208D9224A84F8C150136843F01003B4
:10B720001360FFF756B9D4F89830013BC4F898304D
:10B73000FFF74FB91B4B002283F89420FFF749B95C
:10B74000FF2E7FF449A9194E42B300244FF006089A
:10B750001827687818FB00410138784300F5D3605A
:10B7600000EB8400042206EB81010134FDF719FB94
:10B77000062CEED1FFF72DB929197819042231448E
:10B780000435FDF70EFB182DF6D11834B4F5FC7F07
:10B790003FF41FA9002504F5D067EDE71824F9E769
:10B7A0006006002078F6FF1F0806002064060020CF
:10B7B0007378142B3FF605ADB278052A1BD8062105
:10B7C00001FB0323A54A52F82320A54B7A601B787E
:10B7D000002B3FF4FEA8A34B1A60A34B2AB91A68AA
:10B7E00042F008021A60FFF7F4B81A6822F0080263
:10B7F0001A60FFF7EEB8FF2A7FF4EEA8974E43B326
:10B8000000244FF006081827687818FB004101381B
:10B81000784300F5D36000EB8400042206EB81013D
:10B820000134FDF7F7FA062CEED1FFF7D2B829194B
:10B830007819042231440435FDF7ECFA182DF6D1BD
:10B840001834B4F5FC7F3FF4C4A8002504F5D06794
:10B85000EDE71824F9E77778142F3FF6B2ACB67805
:10B86000300632D57D4E814F00244FF02008AB7852
:10B870002341D90711D504F0010108FA01F141F083
:10B88000010195F80190C9B2C4F3470002F052FBE0
:10B89000062303FB094946F82900BB7E83B16B7878
:10B8A00073B1062111FB03411820013B584300F5F9
:10B8B000D360042206EB810100EB8400FDF771FAEE
:10B8C0000134062CD3D1FFF784B8052E3FF684A8A7
:10B8D00006F001032021994041F001017008C9B22E
:10B8E00002F028FB614B5D4C9B7E062202FB076643
:10B8F00044F82600002B3FF46CA86B78002B3FF433
:10B9000068A8A87812FB03015A1E1823534303F5B5
:10B91000D363042204EB810102FB0030FDF741FAFE
:10B92000FFF757B872784F4B0A2A0CD8DFE802F0BD
:10B9300006151A1F252D32373C4145004C491A681F
:10B9400009680A441A601A68474B002A3AD11A68F3
:10B9500042F008021A60FFF73CB845491A680968C6
:10B96000521AEFE7424A196812684A43EAE7404927
:10B970001A68096892FBF1F2E4E73D4A1868116819
:10B9800090FBF1F201FB1202DCE739491A68096801
:10B990000A40D7E736491A6809680A43D2E73449AA
:10B9A0001A6809684A40CDE731490A68D2430A60FB
:10B9B000C9E719682E4A1160C5E72D4A1968106851
:10B9C0001860F8E71A6822F008021A60FFF701B859
:10B9D000244B1B68C6F80330FDF726FBFEF7F9BFC2
:10B9E0007378052B3EF6F5AFDFE803F0030A111874
:10B9F0001F261D4A136803F00F031360FEF7E9BF0B
:10BA0000194A136823F010031360FEF7E2BF164AC9
:10BA1000136823F020031360FEF7DBBF124A13689C
:10BA200023F040031360FEF7D4BF0F4A136823F0DE
:10BA300080031360FEF7CDBF0B4A136823F48073B5
:10BA40001360FEF7C6BF71782E293FF6BAAB094ADC
:10BA500002EB8102C2F8CC30FEF7BBBF64060020C7
:10BA60006B0800205C080020600600200C80FF1F8F
:10BA70007808002078F6FF1FC84BC94AD3F8881110
:10BA80001160C84AD3F88C111160D3F89021C3F823
:10BA90009820C54AD3F894111160D3F8982183F8FF
:10BAA000C120D3F89C21C3F8C820D3F8A021C3F843
:10BAB000C42093F8A411BD4A505C08B10120505431
:10BAC000002283F8A821FEF784BF00F0D1FEFEF724
:10BAD00080BF00F0CEFEFEF77CBF00F0DDFEFEF77B
:10BAE00078BF00F0DBFEFEF774BF00F0D8FEFEF773
:10BAF00070BF00F0D5FEFEF76CBFA84B002283F8A4
:10BB00009420FEF766BF72782AB1012A09D0032378
:10BB10003B70FEF75EBFA14B012283F89420FEF735
:10BB200058BFB3F5805FBEF457AF9C4981F89420AD
:10BB3000C1F89830FEF74DBF984A9C48002382F820
:10BB4000C03082F8A83102F1CC044FF0FF3519461D
:10BB500044F82350C15401332F2BF9D1904B82F874
:10BB6000941019608F4BC2F8981019608E4BC2F870
:10BB70009C1082F8C1101960FEF72BBF127D92074E
:10BB80000BD4B3F5805FBEF427AF844A042182F85A
:10BB90009410C2F8AC31FEF71CBF08233B70FEF7CF
:10BBA00018BF7E4B002283F89420FEF712BF2B466D
:10BBB0000022E2540133082BFBD123782372FEF7D5
:10BBC00008BF7378012B19D005D3022B1FD0032394
:10BBD0003B70FEF7FEBE764B01221A70754B764A1B
:10BBE0009B781370754B196800230139013311F8E4
:10BBF000010FD054082BF9D1FEF7EBBE1822FA71D1
:10BC00007B7142220923BA713B71FEF7E2BE684B99
:10BC10006B4801221A70674B674A9B7813700023A8
:10BC200001331918082B11F8091CD154F8D1FEF76B
:10BC3000D0BE7378032B3EF6CCAEDFE803F00210E3
:10BC40001E23564B93F89420FA7193F8C120D3F831
:10BC5000AC31BA711A0A7A713B71FEF7BABE4F4B1A
:10BC600093F89420FA7193F8C120D3F89830BA7100
:10BC70001A0A7A713B71FEF7ACBE494B1B687B60B8
:10BC8000FEF7A7BE474B1B687B60FEF7A2BE72782B
:10BC9000002A7EF49EAEB17800297EF49AAE40F27E
:10BCA000D24293427EF495AE45F2FF70FDF767F8FD
:10BCB000FDF7E2F80120FCF7BBFDFEF78ABE01228A
:10BCC000FEF7E3BD75782DB1012D13D003233B7032
:10BCD000FEF77FBE042204A945F2FB70FDF79AF837
:10BCE000049BD6F803209A4206BF01237B607D6047
:10BCF000FEF76FBEB3782A2B07D10422314945F2F3
:10BD0000FB70FDF74EF8FEF764BE03233B70FEF7B1
:10BD100060BE224CD4F8B401002104F5DC728142EB
:10BD20003EF457AE52F821509D4201F1010520D159
:10BD300002EB8503043B0138814214D3C4F8B401FB
:10BD4000FEF747BE154AD2F8B41109299DBF481C19
:10BD5000C2F8B40102EB8102092394BFC2F8B831E2
:10BD60003B70FEF736BE53F8042F43F8042C013124
:10BD7000E2E72946D3E7094A0023C2F8B43119465D
:10BD800002F5DC7242F8231001330A2BFAD1FEF7D8
:10BD900020BE0A237B60FEF71CBE00BF78F6FF1FA3
:10BDA0005C080020780800206006002008060020BB
:10BDB000600800200C80FF1F610800200880FF1F22
:10BDC000008000005B06002003233B70FEF701BEED
:10BDD0007378812B7EF400AEB378922B7EF4FCADA9
:10BDE000B379A32B7EF4F8AD7379B42B7EF4F4AD64
:10BDF0003379C52B7EF4F0ADF378D62B7EF4ECAD21
:10BE0000FCF7F9FEFCF738FC0446FCF735FC001B98
:10BE10000028B8BF4042B0F57A7FF6DBFCF706FD9C
:10BE2000134B00221A604FF0FF32C3F87021C3F8A1
:10BE30007022C3F87421C3F87422C3F87821C3F8C0
:10BE40007822C3F87C21C3F87C220A4B0A4A1A6084
:10BE50000120FCF7EDFCFEF7BCBD40F2D24293425C
:10BE60007EF4B7AD054B012283F8E021FEF7B1BDAA
:10BE700010E000E00080FF1F7856341278F6FF1FB4
:10BE80002DE9F84F484B494F00241C60484BC7F838
:10BE900098401C60474B87F8C1401C6007F150096F
:10BEA00007F1300A444B454A03EB84134FEA8408F8
:10BEB0001B7E002B45D1424B47F8243049F82430F3
:10BEC0004AF8243004F0010120268E4076B2C4F3F3
:10BED000470B46F0070142F82430C9B2584602F039
:10BEE00029F8384A42F80800374A002546F006018A
:10BEF000A554C9B2584602F01DF8344B43F8080067
:10BF0000334BE0B2E554013402F006FE062CC9D1F1
:10BF1000304A2B462946904642F823100133B3F5A8
:10BF2000807FF9D12C4EB37E43BBF37E53B3737D38
:10BF3000BBB3FCF70BFEA0B3012387F89430BDE838
:10BF4000F88F264B47F82430254B49F82430254BF1
:10BF50004AF82430244BB5E7291909EB05000422DF
:10BF600051440435FCF756FF182DF5D11834B4F5BB
:10BF7000FC7FDAD0002504F5D069EDE71824DFF85E
:10BF80006CA0F7E74FF4FF6440F6D805A4F5FF6115
:10BF90002046042241440434FCF73CFFAC42F5D176
:10BFA000C5E70023C9E700BF5C08002078F6FF1F43
:10BFB000780800206006002008040020E0F6FF1F3B
:10BFC000E9EA000090F6FF1FEB030020380600208E
:10BFD000500600207C0800200C80FF1FF9E90000BB
:10BFE00071EA000041EA0000B9EA0000640600209E
:10BFF000F7B50F4C07460E4694E803008DE80300A2
:10C000000C49C1F803300C4B8A7000220F704E703F
:10C010001A70FEF7BBFA094A217882F8E1119DE80F
:10C020000300636884E80300184603B0F0BD00BF56
:10C0300070080020580600206B08002078F6FF1FCB
:10C04000F7B504461F4A63781370A3785370E378FA
:10C0500093702379937163795371A3791A4D137196
:10C06000E379D3700E4695E80300184B00221A704E
:10C070008DE80300FEF78AFA154B1A786F462B46B7
:10C080009AB9327072702A78B2706A78F270EA796E
:10C090003271AA7972716A79B2712A79F27197E86C
:10C0A000030083E8030003B0F0BD012AF7D109487B
:10C0B000721EF11D10F8014F02F8014F8A42F9D1AA
:10C0C000EDE700BF58060020700800206B08002034
:10C0D0006008002061080020014B93F8E1017047DF
:10C0E00078F6FF1F2DE9F043994B9A4C1B788FB0DF
:10C0F0006BB1994B1B78063BDBB2192B04D8974ADE
:10C1000022FA03F3D90702D4002384F8B03194F85B
:10C11000B031934E5A1E012A51D89249012BCA6858
:10C12000079214BF082307238DF81830327894F84B
:10C13000E2318DF8193000238DF81A30002A33D1FE
:10C140008B688DF82030884B8DF8272019788DF872
:10C15000211059788DF82210D9798DF8231099790A
:10C160008DF8241059791B798DF825108DF826301B
:10C1700006A801F0D9FC002800F02A837B4B1A782E
:10C180009846002A00F01E81794B7A4F1B78013BBC
:10C19000062B00F21381DFE813F0F100F1005801E3
:10C1A0001101110111017F01012AE1D1724801330E
:10C1B00006AA1A44195CD171082BF8D1D8E7032BD1
:10C1C0003DD1337883BBDFF89C81674F98F802003C
:10C1D00098F801503B7805441D447B781D44FB7959
:10C1E0001D44BB791D447B791D443B791D44FCF7FC
:10C1F0007DFA98F80100FCF779FA3878FCF776FABE
:10C200007878FCF773FAF879FCF770FAB879FCF7EC
:10C210006DFA7879FCF76AFA3879EDB2FCF766FACC
:10C220002846FCF763FAA9E7012BA7D1524F002556
:10C23000785D0135FCF75AFA092DF9D19EE7042BF8
:10C240002BD1484FDFF82081B8787D780023012278
:10C250000544154488F8013088F80020C8F80430F7
:10C26000FCF744FA7878FCF741FA98F80000FCF7FC
:10C270003DFA98F80100FCF739FA98F80700FCF746
:10C2800035FA98F80600FCF731FA98F80500FCF743
:10C290002DFAEDB298F80400C0E7072B37D13378B8
:10C2A00053BB304B9F7893F801802F4B8DF8007073
:10C2B0001D785878D9798DF8025047443D449A79D1
:10C2C0008DF80300284493F805C08DF8041001444C
:10C2D00093F804E08DF805200A440CEB0203734444
:10C2E0008DF801808DF806C08DF807E08DF80830D4
:10C2F0006846FCF77DFC41E7012BF9D11E4900237C
:10C300005A5C0DF803200133092BF9D1F0E7082B13
:10C310007FF434AF144A1349002301205370107086
:10C3200053608A7849788DF800200A4402448DF8D9
:10C3300001108DF802008DF803308DF804308DF86F
:10C3400005308DF806308DF807308DF80820CFE7DE
:10C350006A08002078F6FF1F58060020110200022C
:10C36000600800200C80FF1F700800205606002087
:10C3700007060020F103002061080020B24A397846
:10C3800093688DF8303080238DF831308A238DF812
:10C39000323000238DF833308DF834308DF835305D
:10C3A0008DF836108DF8293007218DF82A300AA82B
:10C3B000D3688DF828100B9301F0B6FB00233B7077
:10C3C00088F80030002384F8B031337094F8E031FD
:10C3D00013B10120FCF72CFA06A801F031FB064648
:10C3E000002800F04981994B9DF820201A709DF893
:10C3F00021205A709DF822209A709DF823209A716E
:10C400009DF824205A719DF825201A719DF8262048
:10C41000DA709DF8193084F8E231FCF72DF98C4B75
:10C4200018608C4B00221A709DF81830072B0CBF37
:10C430000123022384F8B03194F894305A1E012A63
:10C440004AD9052B48D0012247E0DFF8FC913B7820
:10C4500099F8020099F8015005440A351D44FCF78B
:10C4600045F999F80100FCF741F98020FCF73EF905
:10C470008A20FCF73BF90020FCF738F90020FCF794
:10C4800035F90020FCF732F9EDB23878FCF72EF9D7
:10C490002846FCF72BF991E76B4A507893788DF892
:10C4A0000C303A788DF80D00802103448DF80E1081
:10C4B0000A338A218DF80F101344002103A88DF848
:10C4C00010108DF811108DF812108DF813208DF8C2
:10C4D0001430FCF78DFB71E700225F4B1A7094F863
:10C4E0009430042B04D1594B19780A0640F173811A
:10C4F00094F8B021082A04D840F25113D340DF0742
:10C5000001D4FEF743F894F8B031092B77D1FCF74A
:10C51000B3F8D4F88830514DC01A00282A68B8BF43
:10C520004042904209D94E4B1A78012A04BF022298
:10C530001A70FCF7A1F8C4F88800FCF79DF8D4F84D
:10C540008C306A68C01A0028B8BF4042904209D9AE
:10C55000434B5A78012A04BF02225A70FCF78CF828
:10C56000C4F88C00FCF788F8D4F89030AA68C01A98
:10C570000028B8BF4042904209D9394B9A78012A25
:10C5800004BF02229A70FCF777F8C4F8900094F880
:10C59000C030A3B394F8A8318BBB314A31481D4653
:10C5A000D15C022940F00B8150F823104E1C00F0A2
:10C5B00005812D4A84F8A4311268C4F888212B4AD9
:10C5C0001268C4F88C21D4F89820C4F89021284A25
:10C5D000C4F898101268C4F8942194F8C120C4F8E3
:10C5E00098210023D4F8C820C4F89C2184F8C130D5
:10C5F000D4F8C420C4F8A021012384F8A83194F809
:10C60000B031092B06D194F89420022A04BF0522E8
:10C6100084F89420D4F8B421002A00F0D980092BA2
:10C6200040F0D68094F89430012B40F0D180D4F8BB
:10C6300098101048002350F823508D4240F0C480D9
:10C64000052384F89430C3E00C80FF1F58060020B7
:10C65000F4050020C00300206B080020A405002082
:10C660000806002044F7FF1F5C080020780800201F
:10C670006006002030F8FF1F03A8FCF74FF80546BE
:10C6800000284ED0FCF762F808B184F8E36194F812
:10C69000E3219DF80C10531CDBB22244092B84F8D3
:10C6A000E33182F8E4117FF41AAF604A94F8E411A0
:10C6B00052780023914284F8E3317FF410AF5C4953
:10C6C0005A5C01331644082BF6B2F9D194F8EC31D8
:10C6D000B34222D1574B94F8E5211A7094F8E62121
:10C6E0005A7094F8E7219A7094F8E8219A7194F8B6
:10C6F000E9215A7194F8EA211A7194F8EB21DA7061
:10C70000FBF7BAFF4C4B4D4A18600023137003220D
:10C7100084F8B02184F8E3318EE6042384F8B03144
:10C72000DDE60AAE3046FCF750FA48B32B46F25C21
:10C7300001331544082BEDB2F9D19DF83020AA42FF
:10C74000ECD13C4B9DF829201A709DF82A205A7094
:10C750009DF82B209A709DF82C209A719DF82D2021
:10C760005A719DF82E201A719DF82F20DA70FBF770
:10C7700083FF314B1860314B00221A70072359E6B2
:10C7800094F89430013B012B3FF6A9AED4F89830D1
:10C79000B3F5805F0ED2FCF7D9F958B1D4F8980000
:10C7A0002449431CC4F89830FCF758FB092384F84B
:10C7B000B03148E6002384F8943090E6D554013334
:10C7C0002F2B7FF4EDAE1AE701339A427FF433AF9B
:10C7D0000FB0BDE8F08394F8B001082804D840F207
:10C7E0005112C240D207F3D4D4F8AC01144DD3F89F
:10C7F00003306970B0F5805F6B6012D20D49FCF7B1
:10C8000019FB0C49D4F8AC01FCF76AFB38B1D4F839
:10C81000AC310133C4F8AC3165232B70D8E7072362
:10C82000FBE707232B7000230BE700BF0C80FF1FE3
:10C830005CF8FF1F58060020FC05002006060020BB
:10C8400070080020704710B5074CFBF715FF2368F0
:10C85000C01AB0F5FA7F05D9044B0222DA60FBF763
:10C860000BFF206010BD00BF7C0C002000F00F40CB
:10C870007047064B5A7832B9D3F80310044B01B90C
:10C8800001221A7070470322024BFAE75806002073
:10C89000E40300207008002070477047704770471D
:10C8A0007047704700000000014B53F820007047AC
:10C8B00068F8FF1F2DE9F74FA94DEB69ABB1A94E01
:10C8C000347894B9FBF7D8FEA74B1B68C01A002830
:10C8D000EB69B8BF4042984207D92046013402F0C4
:10C8E0004FF8062CF9D1012333702B6AABB19F4E60
:10C8F000347894B9FBF7C0FE9D4B1B68C01A002822
:10C900002B6AB8BF4042984207D92046013402F052
:10C9100037F8062CF9D101233370964CFBF7ACFEA7
:10C9200094F8303004EB83039B69C01A0028B8BF29
:10C9300040420A2830DDFBF79FFE074694F830009E
:10C94000202100F00103994041F00101C9B24008E3
:10C9500001F0F0FA94F8308004EB880506466B6B22
:10C96000C31A07EE903AAB69FB1AB8EEE77A07EE06
:10C97000903AF8EEE77AC7EE276A16EE900A04F0CE
:10C98000C9FA75A3D3E9002304F018FB04F0B0FD45
:10C9900044F82800AF616E6394F83000202600F060
:10C9A000010106FA01F141F01501C9B2400801F098
:10C9B000C1FA10F04003054600933DD094F83000D2
:10C9C00000F0010106FA01F1C9B2400801F0B2FA23
:10C9D0000138C0B201280AD994F8300000F00101F2
:10C9E00006FA01F10122C9B2D04001F05BFA94F8D5
:10C9F0003000614B012700EA070120261F5406FA88
:10CA000001F15E4B41F006011F544FF6FF72C9B2AF
:10CA1000F84001F047FA94F8300000EA070106FAFE
:10CA200001F141F007010022C9B2F84001F03AFAE1
:10CA300094F83030524AD75494F83000514F07EBF5
:10CA400080131B69002B67D000F00101202606FA35
:10CA500001F141F00201C9B2400801F06BFA94F80B
:10CA6000303007EB831200281269B8BF4042904271
:10CA700052D9E21892F84C20BAB94FEA530903F0A0
:10CA800001039E4046F01406F6B23146484601F0D6
:10CA900051FA314640F48062484601F003FA94F8B6
:10CAA00030300122234483F84C2094F85260DFF8A0
:10CAB000E0B056B9F0B2FBF7C6FF0BF8060001363E
:10CAC000082EF7D1012384F852302F49DFF8BCA09B
:10CAD00027264FF000094FF002085FFA89F0019114
:10CAE000FBF7B1FF1BF809300199834259D009F1D6
:10CAF0000C030BF8090051F82330022B4AD0032B0A
:10CB000003D0012B4DD100284BD01AF80630012B51
:10CB100008BF0AF8068044E094F83060A31993F83F
:10CB20004C30002BC1D006F001034FEA56092026F5
:10CB30009E4046F01406F6B23146484601F0FAF936
:10CB4000314620F48062484601F0ACF994F8303068
:10CB500000222344A7E700BFFCA9F1D24D62904018
:10CB60000C80FF1F06060020FC050020C0030020EB
:10CB7000F405002068F8FF1FEB030020500600209A
:10CB80000004002008040020A4050020080600205E
:10CB9000BBF8FF1F28B91AF80600012801D10AF8CE
:10CBA000063009F10109B9F1080F06F1010694D127
:10CBB00094F8303015F0010104EB030200F0B98065
:10CBC00092F85B1091B9012182F85B10674A1A4410
:10CBD00092F8242012F0010F08D002211B2211FB31
:10CBE0000323634AD05C012808BFD15494F8303045
:10CBF00015F0020104EB030200F0A98092F8611025
:10CC000091B9012182F86110584A1A4492F82A20F9
:10CC100012F0010F08D00E33554A12F813100129F3
:10CC200004BF022102F8131015F0800608D094F812
:10CC300030304F4A0333D15C012904BF0221D15463
:10CC4000009B43B194F83030494A0F33D15C01293D
:10CC500004BF0221D15494F8300007EB80131B6A03
:10CC6000A3B36D0532D400F00101202505FA01F1CE
:10CC700041F01901C9B2400801F05CF9804694F80E
:10CC8000300000F0010105FA01F141F00101C9B2E3
:10CC9000400801F04FF994F8303007EB8317A8EB08
:10CCA000000000283A6AB8BF404290420ED91846A8
:10CCB00001F066FE94F830302E4A0121D15415332C
:10CCC0002B4AD15C012904BF0221D154A6B12A49C3
:10CCD00094F830300A7842FA03F0C0070CD50120EE
:10CCE000264D00FA03F32B70254D28702548007857
:10CCF00010B922EA03030B7094F83000202100F0F1
:10CD00000103994041F01501C022C9B2400801F069
:10CD1000C9F894F8300000F075F894F83030013319
:10CD2000DBB2052B88BF002384F8303003B0BDE8A8
:10CD3000F08F92F85B0000283FF458AF82F85B1048
:10CD40000A4A1A4492F8242012F0020F44E792F89B
:10CD5000610000283FF468AF82F86110034A1A446A
:10CD600092F82A2012F0020F54E700BFA405002019
:10CD700008060020E5030020F2030020F103002054
:10CD800056060020DC0300202DE9F3411A4C235CF9
:10CD900006460F4600F0010845086BB12021174BED
:10CDA00001FA08F141F0060153F82020C9B22846E3
:10CDB00001F078F80023A355202404FA08F4EDB21A
:10CDC00044F0070187EAE772A2EBE7722846C9B28E
:10CDD00001F068F80A4B0122002F9A554FF000032A
:10CDE000D8BF02220192E1B200931A46284600F011
:10CDF000FFFF02B0BDE8F081500600203806002099
:10CE0000EB0300202DE9F04F202100F00106B14096
:10CE10004EB24FEA500A46F015010446C9B287B037
:10CE200050469B4D01F086F84FEA841B05EB0B073B
:10CE30000146387A7F6810F0400F4FEA510201F046
:10CE4000010325D002F00109DAB255F80B305B423C
:10CE500004937B42039310F0800F00F03F0805918C
:10CE6000029220461DD001F0B5FD029A0599B0FA54
:10CE700080F35B0908F1FF3007285DD8DFE810F088
:10CE80001900190019001900810281028102810232
:10CE90005FFA83F955F80B30049302F0010203970F
:10CEA000D9E701F097FD031C18BF01230599029AE9
:10CEB000E0E778480290035D013B0E2B3CD8DFE8A9
:10CEC00013F00F003E005F006C008F00A800C90047
:10CED000F1005401BF01C5013B0026023F022B02B5
:10CEE000DFF8B891DFF8B8A100262027F0B284421D
:10CEF00008D005EB0B035B7E9BB105EB8612527EDF
:10CF00009A420ED100F0010107FA01F141F014013B
:10CF1000C9B2400801F00EF8012349F8260006F8CE
:10CF20000A300136062EE1D1A8F10208B8F1010F4E
:10CF300031D80223029A135507B0BDE8F08F029B47
:10CF400003EB840346F014019A68C9B242F002026E
:10CF5000504600F0A7FF0026AB44F0B2844207D051
:10CF60009BF819303BB105EB8612527E9A4202D1F2
:10CF70000499FFF709FF0136062EEED10323D9E706
:10CF8000002AD9D046F00101C9B2504600F0D2FFC4
:10CF9000414B43F824000423CCE7029B03EB8403BA
:10CFA00046F014019A68C9B242F00102504600F0FE
:10CFB00079FF049B00265F42AB44F0B2844207D065
:10CFC0009BF819303BB105EB8612527E9A4202D192
:10CFD0003946FFF7D9FE0136062EEED10523A9E723
:10CFE000B9F1000FA8D00026AB44F3B2A34207D09A
:10CFF0009BF819303BB105EB8612527E9A4202D162
:10D00000304601F0BDFC0136062EEED1029B1E55C6
:10D0100092E7029B03EB840346F014019A68C9B2BD
:10D0200022F00302504600F03DFF0026AB44F0B270
:10D03000844207D09BF819303BB105EB8612527E33
:10D040009A4202D10399FFF79FFE0136062EEED1D8
:10D0500007236FE7B9F1000F7FF46EAF039BAB447A
:10D060005E425FFA89F0844207D09BF819303BB1E9
:10D0700005EB8912527E9A4202D13146FFF784FEB7
:10D0800009F10109B9F1060FEBD1082352E700BFFE
:10D0900008040020D0F8FF1FC4030020D8F8FF1FA9
:10D0A000EB030020B9F1000F3FF446AF46F0010159
:10D0B000C9B2504600F03EFF0026804605EB0B0744
:10D0C000F0B2844206D07B7E3BB105EB8612527EE5
:10D0D0009A4202D10021FFF757FE0136062EEFD10A
:10D0E000BC4A52F82430A3EB080342F8243000264F
:10D0F0005FFA86F94C4508D005EB0B035B7E7BB3EA
:10D1000005EB8612527E9A422AD14FEA5907202314
:10D1100009F0010903FA09F9AF4B4FFA89FA53F8FC
:10D1200026204AF0140122F00302C9B2384600F06A
:10D13000B9FE4AF00701039AC9B2384600F0B2FEC0
:10D140004AF00D014246C9B2384600F0ABFE00235A
:10D15000019300931A465FFA89F1384600F048FEC1
:10D160000136062EC4D10923E4E689057FF5E4AE35
:10D1700046F00101C9B2504600F0DCFE974B002694
:10D18000186005EB0B07F0B2844206D07B7E3BB102
:10D1900005EB8612527E9A4202D10021FFF7F4FD80
:10D1A0000136062EEFD105EB0B0300274FF0200AC6
:10D1B0000493FEB2B44207D0049B5B7E03B305EB3D
:10D1C0008712527E9A421BD14FEA560906F0010699
:10D1D0000AFA06F676B246F00D010022C9B24846B8
:10D1E00000F060FE46F001010022C9B2484600F09E
:10D1F00059FE46F019010022C9B2484600F052FE1D
:10D200000137062FD5D1A8F10308B8F1010F00F2BC
:10D210008180039B00265F42AB44F0B2844207D07A
:10D220009BF819303BB105EB8612527E9A4202D12F
:10D230003946FFF7A9FD0136062EEED10A2379E61D
:10D24000B9F1000F3FF478AE0B2373E6B9F1000F8C
:10D250007FF472AE46F00101C9B2504600F06AFE9A
:10D2600005EB0B0706465FFA89F0844206D07B7E09
:10D270003BB105EB8912527E9A4202D10021FFF7A1
:10D2800083FD09F10109B9F1060FECD1DFF848A1DE
:10D290000223002796FBF3F30493FEB2B44208D0B6
:10D2A00005EB0B035B7E6BB305EB8712527E9A4254
:10D2B00028D14FEA5608202306F0010603FA06F6A5
:10D2C0004FFA86F95AF8272049F0140122F0030298
:10D2D000C9B2404600F0E6FD49F00701039AC9B221
:10D2E000404600F0DFFD49F00D01049AC9B2404606
:10D2F00000F0D8FD0023019300931A46F1B2404696
:10D3000000F076FD0137062FC7D10D2312E68A05FE
:10D310007FF512AE0E230DE60026AB44F0B2844238
:10D3200007D09BF819303BB105EB8612527E9A422A
:10D3300002D10021FFF728FD0136062EEED1E9E7E4
:10D34000254F00264FF02008AB44F0B2844207D0AE
:10D350009BF8193083B105EB8612527E9A420BD1AD
:10D3600000F0010108FA01F141F0140157F82620FC
:10D37000C9B2400800F096FD0136062EE5D1002323
:10D38000D8E5174F385D01380E283FF6D5AD0FF2BE
:10D39000080E5EF820F000BFE5D300003BD400008B
:10D3A0009DD40000BBD4000021D5000039CF00007F
:10D3B00043D5000039CF000039CF0000EFD5000081
:10D3C0000BD6000097D50000BDD6000069D700003D
:10D3D0003FD70000C4030020D8F8FF1F8C050020B1
:10D3E000D0F8FF1FDFF8D09200264FF0010AF0B20C
:10D3F000844208D005EB0B035B7E9BB105EB8612E4
:10D40000527E9A420ED100F001032021994041F052
:10D41000140106F809A0C9B2400800F08BFDA54B25
:10D4200043F826000136062EE1D1B8F1060F02D0EE
:10D43000B8F1080F3AD1022323E0B8F1060F22D148
:10D4400007EB840346F014019A6822F0030242F0CD
:10D450000202C9B2504600F025FD0026AB44F0B2EE
:10D46000844207D09BF819303BB105EB8612527EFF
:10D470009A4202D10499FFF787FC0136062EEED1BD
:10D4800003233B5558E5B8F1080FE6D107EB8403B9
:10D4900046F014019A6822F00302DAE7A8F10501C8
:10D4A000012905D822B1B8F1060F43D10423E8E7DA
:10D4B000002B3FF441AD0C23E3E7B8F1050F24D175
:10D4C00007EB840346F014019A6822F0030242F04D
:10D4D0000102C9B2504600F0E5FC049B0026C3F1EE
:10D4E0000008AB44F0B2844207D09BF819303BB13E
:10D4F00005EB8612527E9A4202D14146FFF744FC68
:10D500000136062EEED10523BBE7B8F1070FE4D1B3
:10D5100007EB840346F014019A6822F00302D8E76F
:10D52000A8F10502012A07D8B9F1000F04D0B8F11B
:10D53000050F80D00F23A4E7002B3FF4FDAC072399
:10D540009FE7002B7FF4F8ACA8F10708B8F1010FB2
:10D550000CD907EB840346F014019A6822F0030209
:10D5600042F00202C9B2504600F09CFC0026AB44D7
:10D57000F0B2844207D09BF819303BB105EB86121C
:10D58000527E9A4202D10399FFF7FEFB0136062E26
:10D59000EED10A2375E7002B7FF4CEACA8F1070883
:10D5A000B8F1010F0CD907EB840346F014019A6817
:10D5B00022F0030242F00102C9B2504600F072FCB0
:10D5C000039B0026C3F10008AB44F0B2844207D0AD
:10D5D0009BF819303BB105EB8612527E9A4202D17C
:10D5E0004146FFF7D1FB0136062EEED1D1E7002BE5
:10D5F0003FF4A2AC46F00101C9B2504600F09AFCDB
:10D6000007EB840318620B233BE7002B7FF494ACF9
:10D6100046F00101C9B25046049300F08BFC049B14
:10D6200002901E4607EB840304935FFA86F94C458B
:10D6300009D005EB0B035B7E002B35D005EB861282
:10D64000527E9A4230D14FEA5908202309F001094D
:10D6500003FA09F9174B4FFA89FA53F826204AF0D2
:10D66000140122F00302C9B2404600F01BFC4AF04C
:10D670000701039AC9B2404600F014FC049B1A6AE1
:10D68000029B4AF00D011A44C9B20223404692FBA4
:10D69000F3F200F007FC0023019300931A465FFAAF
:10D6A00089F1404600F0A4FB0136062EBDD10D23C2
:10D6B000E7E600BFD8F8FF1FEB0300208B057FF5DE
:10D6C0003BAC46F001010E23C9B250463B5500F079
:10D6D00031FC374B002718604FF02008AB44FEB2F6
:10D6E000B44207D09BF8193023B305EB8712527E62
:10D6F0009A421FD14FEA5609304606F0010608FA51
:10D7000006F676B20021FFF73FFB46F00D0100223E
:10D71000C9B2484600F0C6FB46F001010022C9B27A
:10D72000484600F0BFFB46F019010022C9B2484646
:10D7300000F0B8FB0137062FD1D1FFF7FDBB002663
:10D74000AB44F0B2844207D09BF819303BB105EBF3
:10D750008612527E9A4202D10021FFF715FB013654
:10D76000062EEED10E238CE6DFF8488000264FF01F
:10D77000200905EB0B0AF0B2844207D09AF8193061
:10D7800083B105EB8612527E9A420BD100F0010163
:10D7900009FA01F141F0140158F82620C9B24008F5
:10D7A00000F080FB0136062EE5D1002369E600BFBC
:10D7B0008C050020D8F8FF1F024B1A5C0AB9012221
:10D7C0001A547047D0F8FF1F024B1A5C0AB10F229F
:10D7D0001A547047D0F8FF1F014B185C704700BF08
:10D7E000D0F8FF1F0C4A116940F273234B434FF6E8
:10D7F000FF71B3FBF1F36E2B06D9084B4FF4802178
:10D8000059605723136070474F2B9EBF034B4FF453
:10D8100080219960F5E700BF00B0034080F00F4021
:10D820001B4B1A6802F01F02072A2ED8DFE802F00D
:10D83000040B2D11171D23291A69164992B20A806B
:10D8400041221A6070471A69124992B24A804322F3
:10D85000F7E71A690F4992B2CA804422F1E71A69C0
:10D860000C4992B20A814522EBE71A69094992B242
:10D870004A814622E5E71A69064992B28A8147221F
:10D88000DFE71A69034992B2CA814022D9E700BF93
:10D8900000B00B4008F9FF1F38B541F23001114BC1
:10D8A0005A5842F000625A5041F23C0100245A5842
:10D8B00042F000625A5003F5E8230C2540229D6097
:10D8C0004920DC605C621A6001F016FA064B5722B0
:10D8D0009D602720DC605C621A60BDE8384001F082
:10D8E0000BBA00BF0070044000B003400B2829D8D9
:10D8F000DFE800F0060A0D102828282813281E2328
:10D90000114B188980B270470F4B5889FAE70E4BBC
:10D910009889F7E70C4BD889F4E70B4B588883B20A
:10D9200040F2732058434FF6FF7390FBF3F07047BB
:10D93000054BD88883B28E20F4E7034B188883B256
:10D940004220EFE70020704708F9FF1F30B52E4D49
:10D9500041F23C042B5943F010032B512B4B4FF455
:10D9600000741C636FF4F8755C63A3F51433A4F1C1
:10D970003E542C441C604FF400545C60244C1C60EA
:10D980001C68E401FCD50138072834D8DFE800F032
:10D99000312F2D2B293327041E4858601E4B0020A1
:10D9A00058631E4818601E484FF0806400EA8145A5
:10D9B000C3F88040C3F88450FAB100EA8240C3F84B
:10D9C0009040C3F894004FF08460C3F8A000C3F8FF
:10D9D000A410AAB1C3F8B000C3F8B42030BD1148F8
:10D9E000DBE71148D9E71148D7E71148D5E71148D7
:10D9F000D3E71148D1E71148CFE7C3F89020E2E719
:10DA0000C3F8B02030BD00BF007004400090044057
:10DA10000F0080508720FE01004002400F00800070
:10DA20000000FC1F8720FE038720FE0F8720FE13C7
:10DA30008720FE278720FE638720FEC78720FE07FA
:10DA4000384AD2F88030C3F30363022B5FD0D2F898
:10DA50009030C3F30363022B5BD0D2F8A030C3F342
:10DA60000363022B06D0D2F8B030C3F30363022B5A
:10DA700056D103231B0103F1402202F50032D2F8F4
:10DA80008010C1F303410170D2F8801011F48011AD
:10DA900018BF01218170D2F8801011F4001118BF55
:10DAA000012141704178B1BBD2F88410C1F38A41A1
:10DAB00003F1402303F500334160D3F88810090EC9
:10DAC0000172D3F88810090C4172D3F88810090A42
:10DAD0008172D3F88810C172D3F88C10090E0173CB
:10DAE000D3F88C10090C4173D3F88C10090A817398
:10DAF000D3F88C30C373D2F880309B024CBF4FF008
:10DB000084634FF08063C2F88030012070470023A7
:10DB1000B0E70123AEE7D2F8841021F06041C7E7F7
:10DB20000020704700400240184AD2F87031C3F319
:10DB300003630C2B10B527D04478436804B3C3F3B8
:10DB40001103C2F874318368104A1BBAC2F87831E5
:10DB5000C3681BBAC2F87C318378002C14BF4FF025
:10DB600042624FF040620BB142F4801203781B0412
:10DB700003F470231343054A0120C2F8703110BD2D
:10DB8000034901EA8343DCE7002010BD0040024066
:10DB90000000FC1F0B4B4FF00062C3F870214FF4E4
:10DBA0008022C3F87421084AC3F878216FF4847185
:10DBB000A2F166320A44C3F87C21044AC3F87021FA
:10DBC000704700BF00400240785634120000080C35
:10DBD00010B53A4BDA7842F00202DA70384A10781F
:10DBE000C0B20228114641D0032835D0012832D1D5
:10DBF000546891688C4215D2D978C90707D4516806
:10DC0000D0684C1C5460425CD2B21A7110BD997835
:10DC100001F0DF019970997801F0EF0199701074AB
:10DC2000002317E0517C01F0FF0049B9997801F019
:10DC3000DF019970997801F0EF019970107010BDB3
:10DC4000997841F004019970917CC9B2197100234F
:10DC500053740323137010BD997801F0EF0199708C
:10DC60001B795169DBB20B700223F3E79469D06929
:10DC700084421DD2D2698869121A012A05D19A7884
:10DC800002F0DF029A7000230B70CB698A699B1A3D
:10DC9000022B9FBF094A937843F0080393708A6967
:10DCA0004869531C8B61054B1B79DBB2835410BD53
:10DCB000997801F0DF019970B2E700BF007006406B
:10DCC0001CF9FF1F41F234020A498B5843F08003CC
:10DCD0008B50094B4FF418729A62DA6203F5E03305
:10DCE0001B225A70C0229A7000225A71192001F02A
:10DCF00003B800BF0070044000B0044010B5104BE2
:10DD000000241C745C749A6001225C601A700D4AD5
:10DD1000D960917801F0F7019170917841F010018C
:10DD20009170917800F0FE0041F020019170107127
:10DD30001A78002AFCD1187CB0FA80F0400910BD96
:10DD40001CF9FF1F0070064010B5104B00241C7416
:10DD50005C74DA6103229C611A700D4A59619178F2
:10DD600001F0F7019170917841F010019170917874
:10DD700040F0010041F02001917010711A78002AE2
:10DD8000FCD1187CB0FA80F0400910BD1CF9FF1FCF
:10DD90000070064070B5144C002563610126049B99
:10DDA00025746674A2606560E36140EA0603A561BC
:10DDB000A3740E4BE16026709A7802F0F7029A7015
:10DDC0009A7842F010029A709A7800F0FE0042F0C1
:10DDD00020029A7018712378002BFCD1207CB0FAB5
:10DDE00080F0400970BD00BF1CF9FF1F00700640A5
:10DDF0002DE9F74F01F07F0493461502352C4FEAC9
:10DE00004402984682469DF830709DF83460234B5A
:10DE1000019201D0552C17D148EA050547EA05279C
:10DE20006200224446EA0726924426F4736626F0EE
:10DE30000306F60453F82A20F60C22EA060643F8F5
:10DE40002A6003B0BDE8F08F154A019332F81090B4
:10DE500041F0800100224846FAF722FF002259468D
:10DE60004846FAF71DFF002241464846FAF718FFD8
:10DE7000394600224846FAF713FF31460122484648
:10DE8000FAF70EFF48EA05056300234447EA052731
:10DE90009A4446EA0726019BD1E700BF3CF9FF1FE1
:10DEA000581B01002DE9F84301F07F06352E81460D
:10DEB0001546DFF87C804FEA460401D0552E0FD17D
:10DEC00034444C4425F4736525F0030558F8243098
:10DED000ED04ED0C23EA050348F82430BDE8F8838F
:10DEE000124B33F81070002241F080013846FAF7E7
:10DEF000D7FE0022290E3846FAF7D2FE344400221B
:10DF0000C5F307413846FAF7CBFE4C440022C5F36F
:10DF100007213846FAF7C4FE0122E9B23846FAF77B
:10DF2000BFFE48F82450BDE8F88300BF581B01002D
:10DF30003CF9FF1FF8B5334B01F07F055A1906462F
:10DF4000127B002A56D033F810700022294638463A
:10DF5000FAF7A6FE002211463846FAF7A1FE002283
:10DF600011463846FAF79CFE002211463846FAF769
:10DF700097FE012200213846FAF792FE0022114650
:10DF80003846FAF78DFE002211463846FAF788FE29
:10DF90000022114604023846FAF782FE002211469A
:10DFA00004433846FAF77CFE240204430122002190
:10DFB0003846FAF775FE2402352D40EA040001D0F8
:10DFC000552D0ED105EB45030F4A1E4452F826305D
:10DFD00023F4736323F00303DB04DB0C184342F8E0
:10DFE0002600222D01D0422D0AD1030208D540F08F
:10DFF0007F40F8BD05EB45050544034B53F825006C
:10E00000F8BD00BF581B01003CF9FF1FF8B50E4DCD
:10E0100005440E4695F8003693B9040104F0100447
:10E02000470844F06C0421463846FFF783FF06F0AA
:10E030000F0320F00F021A4321463846FFF732FF44
:10E0400085F80666F8BD00BF3CF9FF1F70B50401F6
:10E0500004F01004460844F06C040D463046214696
:10E06000FFF768FF2D0105F0700520F070022A43CC
:10E0700021463046BDE87040FFF714BF70B504017B
:10E0800004F01004460844F06C040D463046214666
:10E09000FFF750FFED0305F4C03520F4C0322A43EA
:10E0A00021463046BDE87040FFF7FCBE70B5040164
:10E0B00004F01004460844F06C040D463046214636
:10E0C000FFF738FF2D0505F4700520F470022A4390
:10E0D00021463046BDE87040FFF7E4BE70B504014C
:10E0E00004F01004460844F06C040D463046214606
:10E0F000FFF720FF2D0605F0706520F070622A43BF
:10E1000021463046BDE87040FFF7CCBE70B5040133
:10E1100004F01004450844F06C040E4628462146DD
:10E12000FFF708FF3EB140F0804221462846BDE897
:10E130007040FFF7B7BE20F08042F6E770B50401EB
:10E1400004F01004450844F06C040E4628462146AD
:10E15000FFF7F0FE3EB140F4002221462846BDE81C
:10E160007040FFF79FBE20F40022F6E770B504016F
:10E1700004F01004450844F06C040E46284621467D
:10E18000FFF7D8FE3EB140F4802221462846BDE884
:10E190007040FFF787BE20F48022F6E770B50401D7
:10E1A00004F01004450844F06C040E46284621464D
:10E1B000FFF7C0FE3EB140F4804221462846BDE84C
:10E1C0007040FFF76FBE20F48042F6E770B504019F
:10E1D00004F01004450844F06C040E46284621461D
:10E1E000FFF7A8FE3EB140F4005221462846BDE8A4
:10E1F0007040FFF757BE20F40052F6E770B50401F7
:10E2000004F01004450844F06C040E4628462146EC
:10E21000FFF790FE3EB140F4805221462846BDE80B
:10E220007040FFF73FBE20F48052F6E770B504015E
:10E2300004F01004460844F06C040D4630462146B4
:10E24000FFF778FE2B0748BF20F070004FEA051259
:10E250004CBF40F4006020F4076002F070020243FB
:10E2600021463046BDE87040FFF71CBE70B5040182
:10E2700004F01004460844F06C040D463046214674
:10E28000FFF758FEED0105F4F06520F4F0622A4333
:10E2900021463046BDE87040FFF704BEFFF7E6BFF9
:10E2A00070B5040104F01004450844F06C040E46F7
:10E2B00028462146FFF73EFE3EB140F4003221469B
:10E2C0002846BDE87040FFF7EDBD20F40032F6E7C8
:10E2D00008B5094B034493F8002652B9010101F037
:10E2E000100141F06C014008FFF724FE00F00F0020
:10E2F00008BD93F8060608BD3CF9FF1F010108B5EB
:10E3000001F0100141F06C014008FFF713FEC0F36B
:10E31000021008BD010108B501F0100141F06C01C7
:10E320004008FFF707FEC0F3C13008BD010108B582
:10E3300001F0100141F06C014008FFF7FBFDC0F354
:10E34000035008BD010108B501F0100141F06C0156
:10E350004008FFF7EFFDC0F3036008BD010108B5F9
:10E3600001F0100141F06C014008FFF7E3FDC0F33C
:10E37000807008BD010108B501F0100141F06C0189
:10E380004008FFF7D7FDC0F3C04008BD010108B544
:10E3900001F0100141F06C014008FFF7CBFDC0F324
:10E3A000804008BD010108B501F0100141F06C0189
:10E3B0004008FFF7BFFDC0F3803008BD010108B57C
:10E3C00001F0100141F06C014008FFF7B3FDC0F30C
:10E3D000403008BD010108B501F0100141F06C01A9
:10E3E0004008FFF7A7FDC0F3003008BD010101F0B0
:10E3F000100108B541F06C014008FFF79BFDC0F328
:10E400000213020548BF43F00803184608BD010186
:10E4100008B501F0100141F06C014008FFF78AFDDA
:10E42000C0F3C31008BDFFF7F2BF010108B501F04A
:10E43000100141F06C014008FFF77CFDC0F3404043
:10E4400008BD70B5040104F01004460844F06D04E2
:10E450000D4630462146FFF76DFD6D0105F0600564
:10E4600020F060022A4321463046BDE87040FFF7A5
:10E4700019BD70B5040104F01004460844F06D04A1
:10E480000D4630462146FFF755FD6D0305F4C045A6
:10E4900020F4C0422A4321463046BDE87040FFF7D1
:10E4A00001BD70B5040104F01004460844F06D0489
:10E4B0000D4630462146FFF73DFD2D0205F47065FF
:10E4C00020F470622A4321463046BDE87040FFF7D1
:10E4D000E9BC70B5040104F01004460844F06D0472
:10E4E0000D4630462146FFF725FD05F00F0520F0CB
:10E4F0000F022A4321463046BDE87040FFF7D2BCE8
:10E5000070B5040104F01004450844F06D040E4693
:10E5100028462146FFF70EFD20F47F0040EA064220
:10E5200021462846BDE87040FFF7BCBC70B5040129
:10E5300004F01004450844F06D040E4628462146B8
:10E54000FFF7F8FC3EB140F4004221462846BDE802
:10E550007040FFF7A7BC20F40042F6E770B5040155
:10E5600004F01004450844F06D040E462846214688
:10E57000FFF7E0FC3EB140F0807221462846BDE83E
:10E580007040FFF78FBC20F08072F6E7010108B5FC
:10E5900001F0100141F06D014008FFF7CBFCC0F322
:10E5A000411008BD010108B501F0100141F06D01F5
:10E5B0004008FFF7BFFCC0F3413008BD010108B5BA
:10E5C00001F0100141F06D014008FFF7B3FCC0F30A
:10E5D000032008BD010108B501F0100141F06D01F3
:10E5E0004008FFF7A7FC00F00F0008BD010101F093
:10E5F000100108B541F06D014008FFF79BFC0314C2
:10E60000D8B21B0648BF60F0FF0008BD010108B585
:10E6100001F0100141F06D014008FFF78BFCC0F3E1
:10E62000C03008BD010108B501F0100141F06D01D5
:10E630004008FFF77FFCC0F3006008BD10F0010F39
:10E6400070B514BF1826102645080C4628463146DA
:10E65000FFF770FC04F0030420F4401242EA045275
:10E6600031462846BDE87040FFF71CBC10F0010F92
:10E6700070B514BF1825102544080E4620462946BB
:10E68000FFF758FC3EB140F4802229462046BDE801
:10E690007040FFF707BC20F48022F6E710F0010F6E
:10E6A00070B514BF1826102645080C46284631467A
:10E6B000FFF740FC04F0030420F4403242EA044235
:10E6C00031462846BDE87040FFF7ECBB10F0010F63
:10E6D00070B514BF1825102544080E46204629465B
:10E6E000FFF728FC20F47F4040EA06222946204616
:10E6F000BDE87040FFF7D6BB10F0010F70B514BF36
:10E700001825102544080E4620462946FFF712FC1E
:10E7100020F0FF0046EA000229462046BDE870408E
:10E72000FFF7C0BB10F0010F08B514BF182110216E
:10E730004008FFF7FFFBC0F3015008BD10F0010FC8
:10E7400008B514BF182110214008FFF7F3FBC0F3F0
:10E75000804008BD10F0010F08B514BF182110212A
:10E760004008FFF7E7FBC0F3014008BD10F0010FC0
:10E7700008B514BF182110214008FFF7DBFBC0F3D8
:10E78000072008BD10F0010F08B514BF1821102193
:10E790004008FFF7CFFBC0B208BD10F0010F08B56D
:10E7A00014BF192111214008FFF7C4FBC0B208BDF6
:10E7B0002DE9F743F9F760FF0446F9F75DFF001B09
:10E7C0000028B8BF40420928F7DD0026B046F4B261
:10E7D00001254FF035092B4600226C2120461427D5
:10E7E0008DE82002FFF704FB07230022302120469A
:10E7F000CDF804800097FFF7FBFA2B4600227C211E
:10E8000020468DE82002FFF7F3FA0723002250216B
:10E8100020468DE88001FFF7EBFA002211462046E2
:10E82000FFF740FB002220212046FFF73BFB0022A0
:10E830002D212046FFF736FB002221212046FFF73D
:10E8400031FB002240212046FFF72CFB00224D2106
:10E850002046FFF727FB002241212046FFF722FB3D
:10E860002A4623212046FFF71DFBDC2224212046D7
:10E87000FFF718FB46F6DB0225212046FFF712FBC7
:10E8800040F2B71226212046FFF70CFB4DF2B712DB
:10E8900027212046FFF706FB40F2B7122821204629
:10E8A000FFF700FBDC222A212046FFF7FBFA0A22B1
:10E8B0002B212046FFF7F6FA2A4643212046FFF790
:10E8C000F1FADC2244212046FFF7ECFA46F6DB029F
:10E8D00045212046FFF7E6FA40F2B71246212046CE
:10E8E000FFF7E0FA4DF2B71247212046FFF7DAFAB8
:10E8F00040F2B71248212046FFF7D4FADC224A2121
:10E900002046FFF7CFFA2E440A224B212046FFF77C
:10E91000C9FA032E7FF45BAF074D0024AE1F2746D4
:10E92000E0B2FFF7D5FCA75528550134062CF7D1E6
:10E9300003B0BDE8F08300BF42FFFF1F38B5074CAE
:10E94000044494F8001641B994F80656FFF75EFBAC
:10E95000012384F8003684F8065638BD3CF9FF1FC1
:10E96000064B034493F8002632B1002293F80616B2
:10E9700083F80026FFF74ABB704700BF3CF9FF1F32
:10E98000124BF7B501271F54114BC0F347061F5414
:10E9900020243840844065B245F00701304600220B
:10E9A000C9B2FFF77FFA45F0060130464FF6FF7215
:10E9B000C9B2FFF777FA0023019700931A46E1B234
:10E9C0003046FFF715FA03B0F0BD00BFEB0300209F
:10E9D0005006002010F0010F08B54FF004014FEA77
:10E9E000500004D0FFF7A6FAC0F3401008BDFFF7AF
:10E9F000A1FAC0F3001008BD002808B50FDB02F033
:10EA000077FA0DA3D3E9002302F002FC41EC100BCE
:10EA100002F0DAFF51EC100B02F06AFD08BD02F0C3
:10EA200067FA05A3D3E9002302F0F2FB41EC100BD7
:10EA300002F036FFEEE700BF34F7FFFF7F84EE3FC2
:10EA400008B502F055FA08A3D3E9002302F0E0FB71
:10EA500041EC100B02F0B8FF51EC100B02F048FD36
:10EA600008BD00BFAFF30080EB1100A2941A5D4017
:10EA7000002808B50FDB02F03BFA0DA3D3E9002311
:10EA800002F09CFA41EC100B02F00AFF51EC100B63
:10EA900002F02EFD08BD02F02BFA05A3D3E90023F6
:10EAA00002F08CFA41EC100B02F08EFFEEE700BF93
:10EAB00034F7FFFF7F84EE3F08B502F019FA08A390
:10EAC000D3E9002302F07AFA41EC100B02F0E8FEE1
:10EAD00051EC100B02F00CFD08BD00BFAFF300803D
:10EAE000EB1100A2941A5D40704700BF00000000C7
:10EAF00038B500242025E0B200F0010105FA01F14B
:10EB000041F01A014FF48032C9B240080134FFF7D6
:10EB1000C9F9062CEFD138BD2DE9F74F5A4E06EB57
:10EB200080164408F36900F0010723B1B6F81A8093
:10EB3000B8F1000F1BD12025BD406DB245F018067D
:10EB4000E4B2F6B231462046FFF7F4F9314620F43C
:10EB500080622046FFF7A6F945F01A014FF4803293
:10EB6000C9B2204603B0BDE8F04FFFF79BB9FFF7ED
:10EB7000E9FBC0F1080008FA00F002F0B9F9F56904
:10EB8000804685EAE570A0EBE570894602F0B0F9B1
:10EB900002460B464046494602F03AFB00223B4BF8
:10EBA00082468B4602F00AFA8946804649EC108B71
:10EBB000684602F08DFD0022002351EC100B02F09C
:10EBC00065FCF8B14046494602F092FC002D4FF03A
:10EBD000200505FA07F56DB245F01806E4B2F6B265
:10EBE00080463146B8BFC0F100082046FFF7A2F9C1
:10EBF000314620F480622046FFF754F945F01A01AF
:10EC00004246ADE768464BEC10AB02F061FD002DCB
:10EC100059EC108BDDE9000121DD02F069FC18A33D
:10EC2000D3E9002306044946404602F0C7F902F042
:10EC30005FFC2025BD406DB245F01807E4B2FFB27D
:10EC4000064339462046FFF775F9394640F480629D
:10EC50002046FFF727F945F01A01324680E702F017
:10EC600047FCC04306A3D3E90023060449464046B7
:10EC700002F0A4F902F03CFCC0F51C501030D8E7BB
:10EC8000000000000088C340080400200000F0409D
:10EC900000F001032021994041F01901C9B2400858
:10ECA000FFF748B900F001022023934043F0190315
:10ECB0000A464008D9B2FFF7F5B800BFFEE74FF0AB
:10ECC000E0210B4A0B4BC1F8083D4CF22053D38195
:10ECD0004DF62813D381138823F001031B041B0C6A
:10ECE0001380D1F8883D43F47003C1F8883D704724
:10ECF0000020054000800000802800F01F014FF038
:10ED000001030F4A04DD8B40C2F88C31D360704799
:10ED1000402804DD8B40C2F888319360704720287A
:10ED200004DD8B40C2F8843153607047404200F0EC
:10ED30001F0058BF41428B40C2F8803113607047BA
:10ED400000E100E0802800F01F024FF001030D49B0
:10ED500003DD9340C1F88C307047402803DD9340B9
:10ED6000C1F888307047202803DD9340C1F8843013
:10ED70007047404200F01F0058BF42429340C1F824
:10ED80008030704700E100E0074B1A78D2B2012AC8
:10ED900002D1222903D15A7001225A7070472129C9
:10EDA000FAD10022F7E700BF48FFFF1F70B51546F4
:10EDB00011B91B4B197070BD022903D1184B0122E8
:10EDC0001A7070BD04291AD1154B5B78012B25D11F
:10EDD0009488402C28BF402400235E1CDBB2A34251
:10EDE00007D300231A4602211846BDE8704000F000
:10EDF00047BF2A68D05C00F0C3F83346EDE703292B
:10EE000006D1074A5378012B08D100239370E9E714
:10EE1000052901BF024B00221A705A7070BD00BF55
:10EE200048FFFF1F10B50446204600F0C1F8002837
:10EE3000FAD110BD704738B50A4C012502460B4681
:10EE400000202946A57000F0F5FA224618B10023EB
:10EE5000A370122038BD937803F0FF00002BFAD185
:10EE600038BD00BF48FFFF1FF8B506460F4600F04B
:10EE7000F4FC0E4B1A78012A16D15B78012B13D1C2
:10EE800000F000F988B10025ECB2A74205D8214670
:10EE90003046BDE8F840FFF7CEBF301900F0D6F895
:10EEA00001350028F0D0F2E70C20F8BD48FFFF1F25
:10EEB00008B540210248FFF7D7FF00F095F808BDDC
:10EEC0004BFFFF1F38B5054600F0A8F80B28044695
:10EED00009D140210548FFF7C7FF28B92846BDE8FA
:10EEE000384000F09BB80024204638BD8BFFFF1F40
:10EEF00070B50C46461E00250CB9284670BD16F8A4
:10EF0000010FFFF7DFFF013C002818BF0B25A4B25B
:10EF1000F2E738B5451E002415F8010F08B9204660
:10EF200038BDFFF7CFFF002818BF0B24F4E707B563
:10EF30000123002200930649064B104600F020FAF8
:10EF4000002814BF1B20002003B05DF804FB00BFA5
:10EF5000ADED000089ED000038B50C46054600F027
:10EF600097F8A0420AD32C440020A54207D000B154
:10EF700038BD15F8010B00F051F8F6E70B2038BD4D
:10EF800010B50A4A117840290ED05378D4180133AD
:10EF9000DBB2402BA07001F101014FF000001170B5
:10EFA00014BF5370507010BD0B2010BDCBFFFF1F5E
:10EFB00010B50C4A117891B192F84230D41801334F
:10EFC000DBB2A4780470402B4FF0000001F1FF3158
:10EFD000117014BF82F8423082F8420010BD0A203E
:10EFE00010BD00BFCBFFFF1F014B1878704700BF5B
:10EFF000CBFFFF1F024B1878C0F14000C0B2704732
:10F00000CBFFFF1F034B00225A7083F842201A7077
:10F01000704700BFCBFFFF1FFFF7F4BF10B50A4AD0
:10F02000117840290ED05378D4180133DBB2402B2D
:10F03000A07001F101014FF00000117014BF537076
:10F04000507010BD0B2010BD0E00002010B50C4AF2
:10F05000117891B192F84230D4180133DBB2A47820
:10F060000470402B4FF0000001F1FF31117014BF0C
:10F0700082F8423082F8420010BD0A2010BD00BF65
:10F080000E000020014B1878704700BF0E000020D2
:10F09000024B1878C0F14000C0B270470E0000204B
:10F0A000034B00225A7083F842201A70704700BF49
:10F0B0000E000020FFF7F4BF70B50546007801F0A0
:10F0C00093F902780023D9B2914207D25C1C03EB7A
:10F0D000830303445E786B789E4227D1174C2B7ACA
:10F0E000342202FB0142D67813B334234B43E21897
:10F0F000907886420CD000F0030204330C2010FB01
:10F1000002302118205C0B894A68497800F090FB96
:10F11000D4F89C3083B12A46287812F8081F0029B9
:10F120000CBF03210521BDE8704018472346CAE7FC
:10F13000937801339370D8E770BD00BF540000206E
:10F140002DE9F04F85B00D4690468DF80F0001F087
:10F150004BF9022D064647D1077800235C1CDBB231
:10F16000BB4210DB4FF00009DFF8B0B0CA465FFACF
:10F1700089F4A74212DC284BD3F89C30002B45D1F0
:10F1800005B0BDE8F08F03EB830333440DF10F00AE
:10F19000DA78597801F0E2F92346DFE704EB8404DA
:10F1A0003444E378A2886178CDF804A0A078009078
:10F1B0000DF10F0001F0B0F9A378032B05D15A46E9
:10F1C00061789DF80F0001F031FA6178E37841F041
:10F1D000100141EAC3110022C9B20DF10F0001F084
:10F1E000EDF909F10109C2E7002DC4D10A490378FC
:10F1F000342000FB03138A1C3633294634329A42EA
:10F20000B9D002F8341C02F8331CF7E7424629460D
:10F210009DF80F009847B3E754000020B9F00000B4
:10F22000F0B40C7804F06004202C1D4632D14C78E8
:10F23000042C1DD00AD8012C04D003D3022C20D0DA
:10F24000032C12D000202880F0BC7047212C1BD04A
:10F2500004D8202CF6D1F0BC00F040B9222C16D0F6
:10F26000232CEFD1F0BC00F049B9F0BC00F049B953
:10F2700002241C801468002525701468671C176020
:10F280006570F0BC00F056B9F0BC00F01FB9F0BCDE
:10F2900000F076B9402C06D1044CD4F8A04014B14B
:10F2A000A446F0BC6047CD20CEE700BF540000204C
:10F2B00073B50446007801F097F863680093A27A6A
:10F2C000637A43EA0223ADF8043002780023D9B20E
:10F2D000914207D25D1C03EB830303445E7863789D
:10F2E0009E4225D1174D237A342202FB0152D67853
:10F2F00003B334234B43EA18907886420CD000F0D5
:10F30000030204330C2010FB02302918285C0B89FF
:10F310004A68497800F08CFAD5F89C3033B1227AEB
:10F3200020785AB104F108020521984702B070BD57
:10F330002B46CCE7937801339370DAE76A460321D2
:10F34000F3E700BF5400002007B543680093437AF9
:10F35000817A43EA0123ADF80430084BD3F89C309E
:10F3600002462BB1017A007829B10832052198476D
:10F3700003B05DF804FB6A460421F8E7540000205E
:10F380002DE9F84305460F461646984601F02CF83D
:10F3900002789DF8203001328146D2B20021284601
:10F3A00001F09EF80446E8B9164A1749284600F0CD
:10F3B00086F999F80000154B342200FB022209F16E
:10F3C00001011A4499463433934201F105010CD1ED
:10F3D0004146284600F074F8044618B9C9F89C70F4
:10F3E000C9F8A0602046BDE8F88311F8050C03F8C1
:10F3F000340C11F8040C03F8330C03F8324C03F806
:10F40000314CE0E721F2000041F1000054000020FF
:10F4100008B5074B0022C3F89C20C3F8A02000F0D9
:10F42000A1F918B9BDE8084001F06EB808BD00BFE9
:10F43000540000202DE9F041984605460E46174637
:10F4400000F0D2FF04780023D9B2A14207D20133E1
:10F4500003EB8302024412F8042CB242F4D1174C9D
:10F4600034234B43E218D07892F802E0A0EB0E016F
:10F47000C9B2042902D1C120BDE8F08100F0030126
:10F480000130C0B24FF00C0C0CFB0133D070A0EB7C
:10F490000E001C44C0B2012825716671A760A4F853
:10F4A0000C8007D143463A4631462846BDE8F04134
:10F4B00000F0BEB90020BDE8F08100BF540000207C
:10F4C000014B002019607047F8000020024B0979B9
:10F4D000197100F08DBF00BFF800002013B50024A3
:10F4E00002AA1C80044B42F8041D0979197100F02E
:10F4F0008DFF02B010BD00BFF80000200020188072
:10F50000704730B40C460221198021796488084D77
:10F51000012C297102D130BC00F08EBF022C02D127
:10F5200030BC00F095BF0020188030BC704700BF91
:10F53000F800002030B40C4602211980217964883B
:10F54000074D012C297102D130BC00F08DBF022C77
:10F5500002D130BC00F09ABF0020188030BC704748
:10F56000F8000020044B054A19795B791171137278
:10F5700003210A23FFF75EBFF80000204C80FF1F25
:10F58000F8B500271F808B780B4CA371C3F34003A1
:10F590005A0063F3000206466271FFF7E3FF256835
:10F5A00045B1A37913F002021ABF3A462221212164
:10F5B0003046A8470020F8BDF8000020034B00F1BA
:10F5C00008021B6800780521184700BF00010020D1
:10F5D00070B5094D04462A1D012100F0D7FF802295
:10F5E0000121204600F0EAFF2B68207800220A2142
:10F5F000BDE87040184700BF0001002037B5012169
:10F600000DF10702044600F0C1FF9DF80730074DD9
:10F61000802B04D12A790121204600F0CFFF2B68EE
:10F62000207800220B21984703B030BD0001002054
:10F63000436805215A7800F0C1BF73B50122002448
:10F6400005460126002100F089FF334621468DE85A
:10F6500050001022284600F05FFF2246214628462F
:10F6600000F07CFF234621468DE8500010222846FA
:10F6700000F052FF31460222284600F09FFF32463A
:10F680000621284600F09AFF22469021284600F0E5
:10F6900095FF044B28781B682246214602B0BDE83E
:10F6A000704018470001002042783AB9C178C9017A
:10F6B00041F0100101F0900100F080BF704773B578
:10F6C0000C468DF8070001F00DFA1F4D2C60044622
:10F6D000002836D11D4A9DF80700102100F0A6FF32
:10F6E0001B4A044612219DF8070000F09FFF194AAB
:10F6F000044314219DF8070000F098FFE4B204438E
:10F70000154A9DF80700132100F090FFE4B204436E
:10F71000124A9DF80700172100F088FF02AEE4B2FC
:10F7200004430F4A16F8010D162100F07FFFE4B2E2
:10F73000044303220121304600F040FF0323E4B2DA
:10F740002B71204602B070BD000100203BF6000086
:10F7500031F60000D1F50000FDF50000A9F600002B
:10F76000BDF5000037B502AD174B05F8010D0022BD
:10F77000102128461A6000F05BFF1221044628463B
:10F7800000F056FF14210443284600F051FFE4B274
:10F7900004431321284600F04BFFE4B20443172131
:10F7A000284600F045FFE4B204431621284600F045
:10F7B0003FFFE4B2204310F0FF0003D19DF80700A3
:10F7C00001F09CF903B030BD000100201FB50121FC
:10F7D0008DF807000DF10E020DF1070000F0D6FEC6
:10F7E0000DF10F0206210DF1070000F0CFFE9DF88C
:10F7F0000E30802B18D19DF80F309B0714D59DF843
:10F80000070000F0EFFD012804460DD172B60DF19E
:10F81000070000F029FB002221460DF107008DF8BA
:10F820000E2000F0CBFE62B69DF80E0004B010BDB5
:10F8300073B50C4615461E468DF80700FFF7C6FF48
:10F84000802808D033462A4621460DF1070000F0F3
:10F85000A7FA02B070BD0020FBE77047062812D857
:10F8600080000129C0B201D10230C0B2074AC0F302
:10F870004703122101FB03231A884FF6FF739A42B4
:10F8800008BFFF207047FF20704700BF080100201D
:10F890002DE9F041314C324D324E4FF0000884F8E2
:10F8A00000814FF4107285F840020F462846FF2170
:10F8B00001F0C0FE4FF4806241463046C5F8446214
:10F8C00001F0B8FE94F80C3143F0800384F80C3159
:10F8D00094F80C311B06FBD4234BFF221A7094F8CA
:10F8E0000C3143F0400384F80C31204B196897B376
:10F8F00041F000411960194B310AC6F3074201F08B
:10F90000FE0183F89C1083F8B020320E83F8B420F7
:10F91000174AC5F84822102283F80821012283F8EB
:10F920009420BF2283F8802093F8002102F07F0208
:10F9300083F8002193F8842042F0010283F88420A8
:10F9400093F8842042F0100283F8842084221A77EE
:10F950000020BDE8F08121F00041CBE70020074006
:10F9600008010020000E00205680FF1F0070044098
:10F97000001000200D4B93F80C2102F0BF0283F819
:10F980000C21BF2283F8802093F8842002F0FE022D
:10F9900083F8842093F8942002F0FE0283F89420E8
:10F9A0001A7F02F07B021A77002070470020074080
:10F9B000F7B5082304248DE81800B1F803300D785A
:10F9C0008878B3F5007F81BF0023CB7002230B71D1
:10F9D000062D71D8AB00DCB2012804BF0234E4B2BA
:10F9E0004FEA540E354C122707FB0E474FF6FF76B1
:10F9F000B7F800C0B4455FD14E78032E5CD801281B
:10FA00005AD897F80FC0BCF1FF0F04BF4FF0000C9D
:10FA100087F80FC0B1F803C0122101FB0EFE04EB02
:10FA20000E0743EA4003BA73FA7B7E7402F00102C8
:10FA300013435BB2D4F84822C7F80220D9B2F97355
:10FA40003874D4F8447224F80EC01BB207EBC30E0E
:10FA500081F00101CEF80420AEF802C04FF0080E8C
:10FA600007F833E007EBC10ECEF80420AEF802C071
:10FA700012FA8CF24FF0480E07F831E0C4F8482231
:10FA800028B917F8332062F07F0207F8332002AA62
:10FA900002EB80002DB20A4950F8082C11F82530ED
:10FAA000012E0CBF164642F001063343DBB201F8CB
:10FAB0002530002003B0F0BD9520FBE708010020B1
:10FAC000C0200740084610B51146FFF7C7FEFF28C3
:10FAD0001DD0104B1221C0F3470001FB0030D3F8BA
:10FAE0004422C37B1CB283F0010312F8341001F0EE
:10FAF0007F0102F8341012F8331001F07F0102F890
:10FB000033104FF0FF338372C372002010BDC42046
:10FB100010BD00BF0801002073B50C468DF807002A
:10FB2000114620461646FFF799FEFF28054620D0CD
:10FB3000214632460DF10700FFF7C4FFC5F3470326
:10FB400012210D4D59436B18D5F848221888121A06
:10FB5000C5F8482224B2094A002002F824004FF0D8
:10FB6000FF326A549A705A70DA701A715A7102B080
:10FB700070BD9620FBE700BF08010020C0200740B1
:10FB80002DE9F0410E468046114630461746FFF7F4
:10FB900065FE0C4DC0F34700122303FB0050C47BED
:10FBA000FF2C0DD03A4631464046FFF78BFF24B27A
:10FBB000D5F8442212F8343063F07B0302F8343075
:10FBC000BDE8F0810801002010B508460021144668
:10FBD000FFF744FE084AC0F34700122101FB002052
:10FBE000D2F84432C27B03EBC2035A681368236025
:10FBF0005368636010BD00BF0801002010B50C46BB
:10FC000020461146FFF72AFEFF281AD024B2104BD7
:10FC100013F82430DBB213F00C0F12D09B0712D470
:10FC20000C4BD3F8443213F83020D2090DD180F0B8
:10FC30000100C0B213F83030DB0914BF03200020EC
:10FC400010BD052010BD012010BD032010BD00BF58
:10FC5000C02007400801002008B5FFF7FFFD074A54
:10FC60001223C0F3470003FB0020C37BFF2B1EBF02
:10FC7000D2F84422002102F8331008BD0801002008
:10FC80002DE9F0410846002190461F46FFF7E6FDAA
:10FC90002249C0F34700122404FB0014E57BFF2D2A
:10FCA00039D022884FF6FF7093B2834233D0D1F817
:10FCB000441285F0010011F9300000282BDB2EB230
:10FCC00087B901EBC60338465A80D4F802205A603F
:10FCD00011F8352002F0400262F0770201F8362078
:10FCE000BDE8F08101EBC602BB424FF0000028BF27
:10FCF0003B466781C4F80680207360735380C2F866
:10FD0000048011F8353003F0400363F0770301F805
:10FD10003630BDE8F0819420BDE8F0810801002074
:10FD20002DE9F0410C460646114620461546FFF7E0
:10FD300095FD194BC0F34700122202FB003090F8EA
:10FD40000FE0BEF1FF0F24D027B2144A6CB1407C03
:10FD5000012D0CBF14211821012818BF41F0010109
:10FD600012F82700014302F8271012F827106FF34A
:10FD7000410102F82710D3F84432002203F83E2054
:10FD80003DB92B462A4621463046BDE8F041FFF7F3
:10FD900077BFBDE8F08100BF08010020C020074008
:10FDA0002DE9F0410C462046012117469846FFF701
:10FDB00055FDFF2836D01C4BC0F34700122202FB32
:10FDC0000030D3F8446290F80FE016F93E30002B73
:10FDD00028DB23B2154A12F8235015F0020521D171
:10FDE0000188C0F806701FFA88F242818A42D8BFA3
:10FDF00011460FFA8EF206EBC20305734573598064
:10FE00005F602CB9C82306F832302046BDE8F08187
:10FE100016F83E3003F0400363F0770306F8323003
:10FE20002C46F2E79324F0E708010020C0200740A9
:10FE3000034B044883F898100122114600F0BEBB22
:10FE40000020074048030020054B0648002283F8A5
:10FE50009420802283F80C210121FF2200F0AEBB08
:10FE6000002007404803002038B51A4C94F80021C0
:10FE700002F07F0284F8002194F80C2102F0DF02E6
:10FE800084F80C2194F8802042F0200284F880202D
:10FE900094F8842002F0DF0284F8842094F89420FF
:10FEA00002F0DF0284F8942094F8942042F00402D7
:10FEB00084F8942044F62065013DADB200F0BCFE0C
:10FEC000002DF9D194F8943003F0FB0384F89430BA
:10FED00038BD00BF002007402DE9F04FD84DD94C68
:10FEE00095F8807095F8843095F8906087B0FF227F
:10FEF0001F4094F840328DF809208DF80C308DF8B1
:10FF00000D20002301210DF1090204F510708DF878
:10FF10000E3004938DF815308DF816308DF80F30B3
:10FF20008DF8143000F032FB95F80C31D907F6B299
:10FF30000FD59DF80930802B0BD195F8003103F0D7
:10FF40007F0385F8003195F80C3103F0DF0385F865
:10FF50000C317A0711D5BA4B042093F8A41093F80A
:10FF6000A02083F8800006AB42EA012223F80E2D80
:10FF700003A91220049300F06DFBFB074BD5B04D95
:10FF8000B0480123BF2685F8803085F8886095F851
:10FF90009430002743F0020385F894304FF4107238
:10FFA00085F89870FF2185F8007101F043FB4FF44C
:10FFB00080623946D4F8440201F03CFBD4F8443264
:10FFC00003F50073C4F848329F4BFF221A7095F86E
:10FFD000943003F0FD0385F8943095F80C3143F02C
:10FFE000400385F80C319F2385F88C6085F88430B8
:10FFF00095F8943003F0DF0385F8943003A91020BE
:020000021000EC
:1000000000F028FB95F8943003F0DF0385F8943076
:1000100007B0BDE8F08F3D0740F19380884B082280
:1000200083F880203309C6F3C000062B8DF80D300D
:100030008DF80F0000F2F480C6F3800202EB830219
:1000400008B10232D2B2D4F8446206EBC201C2F364
:100050004705D1F804E04988ADF81510122101FBDD
:100060000541CDF810E091F80FC08CF0010C81F83B
:100070000FC016F8321082F0010A5FFA8AFAC1F353
:1000800080110FFA8AF881F00101890106EBC80995
:1000900006F83810002800F0D980DFF8ACB19BB921
:1000A0009BF8002082B9FF2219468BF8002003A894
:1000B0001A460193FFF706FD019B06F838301A46F1
:1000C000194603A8FFF7DCFD9BF80030012B04D094
:1000D0009DF80D30002B00F0AD80122101FB054191
:1000E000BDF815008B894A8903449BB293428B81EA
:1000F00009D3B1F800E0C0B2864540F09380897B17
:10010000012940F08F80122101FB0544D4F806102C
:1001100020881944D31A8342D8BF98B2A9F80200A4
:10012000C9F8041016F83A3003F0400363F077037F
:1001300006F83830424A92F8943003F0DF0382F830
:100140009430B80717D53E4C022384F8803094F8D9
:10015000883094F88C2003A9134016208DF81430B1
:1001600000F078FABF2384F8883094F8943003F0D4
:10017000DF0384F89430F9061CD5314C202384F831
:100180008030102384F8803003A9142000F062FA34
:1001900094F80C3143F0200384F80C3194F80031CA
:1001A00043F0800384F8003194F8843043F0200356
:1001B00084F88430BA060DD5214C202384F8803091
:1001C00003A9132000F046FA94F8843003F0DF030B
:1001D00084F884303B067FF51BAF0DF10A02FF2344
:1001E000102103A88DF80D3000F0D0F99DF80A30E9
:1001F000134C012B04BF8DF80F3000224FF0800309
:1002000008BF8DF80D2003A984F88030172000F076
:1002100021FA94F8943003F0DF0384F89430F7E681
:10022000FF2210E7122202FB0544D4F806200492B4
:10023000ADF8153003A99DF80D0000F00BFA79E731
:1002400000200740080100205680FF1F6BB916F8F8
:1002500032202F4902F03C02342A35D101238DF897
:100260000E309EF80030DB090B70122101FB0541B6
:100270004FF6FF734A899A42DCD0BDF815E08B89AE
:1002800073449BB28B8109888E4501D19A420CD868
:100290008AB3B2FBF1F001FB102080B258BB1220F0
:1002A00000FB0540807B012825D1D21A8A42D8BFA5
:1002B00091B2122202FB0544C9B9D4F80230C9F840
:1002C0000430A9F802102DE70A78012ACDD1FF20C9
:1002D0000870194603A80193FFF7F4FB019B06F889
:1002E00038301A46194603A8FFF7CAFCBDE7D4F810
:1002F00006201344E3E7122202FB0544D4F806204B
:10030000ADF815304FF0FF330492A372E37291E71A
:100310005680FF1F13460A46194601F08BB900BFED
:1003200030B50329039C04981DD12BB9164A2260CD
:1003300004220280002030BD40F209418B420FD1DF
:10034000022A4FF000030CD810490C2505FB0313BB
:10035000D9681B6951F8221021609B5C0380E9E792
:1003600001230122F0E7072901D9CD2030BD074B39
:1003700003EB8102126A2260002AF6D003EB4103EC
:10038000B3F84030EAE700BF5780FF1FE41B0100CD
:1003900001299FBF034B5B5C1370002088BFCD20F9
:1003A000704700BF5403002001299DBF024B00206D
:1003B0005A54CD20704700BF5403002019B14B1E82
:1003C00058425841704701207047054B1A788A42BD
:1003D00004D05878431A584258417047012070475A
:1003E000540300200020704700487047341C01006F
:1003F00001299FBF044BC1EBC101C918002094BF64
:100400001160CD20704700BF5B80FF1F012930B510
:100410000ED8084DC1EBC10108231068C45CC81890
:10042000284401330F2B00F8084CF6D1002030BDD2
:10043000CD2030BD5B80FF1F01299FBF034B03EB25
:1004400041010020116088BFCD2070475603002075
:1004500001299FBF034B03EB41010020116088BFBE
:10046000CD2070475A03002001290AD81368187854
:10047000054B03EB4101887013685B78CB7000205B
:100480007047CD20704700BF5403002001290AD8CF
:1004900013681878054B03EB4101887113685B788A
:1004A000CB7100207047CD20704700BF540300205F
:1004B000084B5A7803F8022BFF210022D154013255
:1004C000072AFBD1044A0023052199540133072B45
:1004D000FBD170475E0300206703002000BF704718
:1004E000013AD2B2062A10B51C4608D8054B5A70FC
:1004F000FFF7DEFF2146BDE81040FFF7C9B999209C
:1005000010BD00BF5E030020024B00225A70FFF7AF
:1005100031BA00BF5E03002037B50F4C257805B90E
:10052000C1B98DF802308DF800109DF81830ADF883
:10053000032069469DF81C2000788DF80130FFF7F4
:1005400037FA9DF800301BB110B92378013B2370B6
:1005500003B030BD9520FBE75E03002038B50A4BA1
:100560000D461C7859788C421C4600D14DB929465D
:100570000078FFF7D1FA2DB120B923780133237029
:1005800038BD962038BD00BF5E0300204B1E062BF1
:1005900005D8094B19444B78137000207047CB06DF
:1005A00007D501F00F01062903D8034B19444B7AF4
:1005B000F2E78220704700BF5E0300204B1E062B2F
:1005C0002DE9F0418046174605D8174B19444A706B
:1005D0000020BDE8F081CB0622D501F00F05062DE5
:1005E0001ED8012A4FEAD1140F4E06D122462946C1
:1005F000FFF7C6FA35446F72EAE7002AFAD1731999
:100600005B7A012BF6D122462946FFF789FB002DA4
:10061000F0D184F0010229464046FFF781FBE9E76B
:100620008220BDE8F08100BF5E03002000207047FB
:10063000062903D9A1F11003072B07D8044B53F85F
:100640002130002B0CBFC42000207047C42070470D
:100650005C1C0100102810B50C4601D1FFF728FFE3
:10066000034B53F820300BB120469847002010BDB3
:100670005C1C01001FB5144602228DF807001A8089
:1006800005210DF10F020DF10700FFF77FFF034B6E
:100690009DF80F201A80236004B010BD7003002065
:1006A0001FB5144601228DF807001A8004210DF1B0
:1006B0000F020DF10700FFF769FF044B9DF80F20B3
:1006C0001A800020236004B010BD00BF700300201A
:1006D000F0B5002685B01E8049888DF80700ADF87A
:1006E0000E10FFF76BFE18B3BDF80E20114F04ACCF
:1006F000B2FA82F2520901210DF10700FFF75EFF05
:1007000034F8022D0421D2B20DF10700FFF756FF95
:100710007B682246012105469DF8070098477B68C3
:100720009DF80700324602219847284605B0F0BDE3
:100730000425FAE77003002073B502AC002504F825
:10074000010D0E461D80042201212046FFF736FFD1
:100750007288024B28461A7202B070BD70030020E6
:1007600013B54C8889888DE80C000B46E2B2210A4B
:10077000FFF7D6FD02B010BD2DE9F04186B0174657
:100780001E4606AA00238846059303238DF80F0012
:1007900002F8083D01210DF10F00FFF7F7FE98F870
:1007A0000050274C15F0030528D10DF11102062148
:1007B0000DF10F00FFF7EAFE9DF811309DF80F00D4
:1007C00003F0030323800DF11203019305AB0093A3
:1007D0002A462B460221FFF7A3FD059BDB7913F088
:1007E000400F238814BF43F0010323F0010323804B
:1007F000022333803C6006B0BDE8F081012D08D1B2
:100800009DF81030012B02D198F80430ABB90023C9
:10081000EDE7022DEED198F8041041F010010DF132
:100820001202C9B20DF10F00FFF7B0FE9DF81230B1
:1008300003F0010323803580DCE7CD20DAE700BF39
:10084000700300207FB500221A800B784E788DF857
:10085000070013F003030D46C6F3400634D1FEB182
:100860004B88013B9BB2012B52D80DF10F020621A0
:100870000DF10700FFF78AFE044670B9AB7801223C
:100880009A409DF80F301A43D2B206210DF10700AD
:100890008DF80F20FFF792FE0446204604B070BD8D
:1008A0004E88012E34D10DF10F0206210DF1070003
:1008B000FFF76CFE04460028EFD1AA7896409DF819
:1008C0000F2022EA0602E0E7022B21D109798DF8F8
:1008D0000F10324641F010010DF10700FFF76EFED8
:1008E0006B78002E14BF07210821012B044607D185
:1008F0009DF80F00C10900F00F00FFF7ADF90821C6
:10090000044B9DF807005B680DF10F029847C4E7A0
:10091000CD24C2E77003002010B500241C800B78A2
:1009200003F00303012B05D18A780979FFF73CFD19
:10093000204610BD042010BD38B515460A7802F0D7
:100940000302012A07D1054C1A8009792246FFF7D4
:100950001FFD2C6038BD042038BD00BF700300208F
:1009600013B5CD298DF8070007D1012290210DF193
:100970000700FFF723FE02B010BD0D491C88088A4E
:100980001268844288BF18800C461B889DF80700B7
:100990000021FEF74DFF94F90A30002BEBDA00231B
:1009A0001A4619460DF10700FFF76AF9E3E700BFA1
:1009B0007003002073B5054600266A4601218DF8B4
:1009C00000600196FFF7E2FDAA78434C012A52D15C
:1009D00068680368C4F80A304368A07AC4F80E3027
:1009E00004F10A0110F0600F1ED1E27A3B4B53F87C
:1009F0002240002C3DD09DF80000022839D802EB9F
:100A000042021344034493F83430012B31D10DF1E9
:100A1000020301AA2878A0470DF1020301AA0146AA
:100A20002878FFF79DFF13E0238AADF80230202BD2
:100A300017D87BB102060DD40A68C4F812204A68A0
:100A4000C4F81620314604F11A022846FFF718F9B7
:100A500002B070BDE46B64B10DF1020301AA20493C
:100A6000D8E702A82B7800F8073D9021FFF7A6FDF4
:100A7000EEE7CD20D0E79DF80030042B10D12B7885
:100A8000217A02AD05F8063D2846FFF7D1F901228B
:100A900011462846FFF792FD227A03212846E5E712
:100AA00094F90A30002BD3DBEB78002BD0D1E66B26
:100AB00086B1B5F8093028780833ADF8023004F172
:100AC00012010DF1020301AAB04701460DF1020324
:100AD00001AAA5E7CD21F9E770030020BC1C0100A5
:100AE0007A030020034B5960DA630021024AFFF7C2
:100AF0009DBD00BF70030020B509010007B502AB22
:100B0000054A03F8010D002118465160D163FFF733
:100B10008FFD03B05DF804FB7003002000207047D8
:100B2000354B41F248015A5822F00F0242F00202BE
:100B30005A5041F204015A5842F480225A5041F26C
:100B400034015A5842F480225A5003F52C33602164
:100B500093F8942042F0020283F89420C02283F894
:100B60000021FF221A7483F8802083F8882083F8FC
:100B70008420002283F88C2083F80C111F491A75F9
:100B8000080A00F0FE0083F8982083F8C02083F85C
:100B9000C42083F8C82083F8CC2083F8D02083F8C1
:100BA000D42083F8D82083F8DC2083F8E02083F871
:100BB000E42083F8E82083F8EC2083F8F02083F821
:100BC000F42083F8F82083F8FC2083F89C00C1F31C
:100BD0000740090E83F8B00083F8B41083F8AC2006
:100BE0001A7783F8082193F8942002F0D40242F097
:100BF000010283F89420704700700440000E00202A
:100C0000024B4FF400125A60704700BF00E100E051
:100C1000034B4FF40012C3F884215A60704700BFA1
:100C200000E100E008B5FEF782F910B9FFF7F0FF28
:100C300008BD1B2008BD00BF034B4AF202629A8127
:100C40004BF280429A8170470020054081F00041BC
:100C500002E000BF83F0004330B54FEA41044FEAA1
:100C6000430594EA050F08BF90EA020F1FBF54EA3C
:100C7000000C55EA020C7FEA645C7FEA655C00F0D8
:100C8000E2804FEA5454D4EB5555B8BF6D420CDDA9
:100C90002C4480EA020281EA030382EA000083EA2C
:100CA000010180EA020281EA0303362D88BF30BDCC
:100CB00011F0004F4FEA01314FF4801C4CEA113122
:100CC00002D0404261EB410113F0004F4FEA033381
:100CD0004CEA133302D0524263EB430394EA050F0C
:100CE00000F0A780A4F10104D5F1200E0DDB02FA7B
:100CF0000EFC22FA05F2801841F1000103FA0EF20F
:100D0000801843FA05F359410EE0A5F120050EF1D4
:100D1000200E012A03FA0EFC28BF4CF0020C43FA05
:100D200005F3C01851EBE37101F0004507D54FF012
:100D3000000EDCF1000C7EEB00006EEB0101B1F562
:100D4000801F1BD3B1F5001F0CD349085FEA3000A8
:100D50004FEA3C0C04F101044FEA445212F5800FB3
:100D600080F09A80BCF1004F08BF5FEA500C50F150
:100D7000000041EB045141EA050130BD5FEA4C0C33
:100D8000404141EB010111F4801FA4F10104E9D1BC
:100D900091F0000F04BF01460020B1FA81F308BFB3
:100DA0002033A3F10B03B3F120020CDA0C3208DD7F
:100DB00002F1140CC2F10C0201FA0CF021FA02F15A
:100DC0000CE002F11402D8BFC2F1200C01FA02F1CA
:100DD00020FA0CFCDCBF41EA0C019040E41AA2BFEF
:100DE00001EB0451294330BD6FEA04041F3C1CDAB7
:100DF0000C340EDC04F11404C4F1200220FA04F0D7
:100E000001FA02F340EA030021FA04F345EA030180
:100E100030BDC4F10C04C4F1200220FA02F001FA42
:100E200004F340EA0300294630BD21FA04F02946C4
:100E300030BD94F0000F83F4801306BF81F480115D
:100E40000134013D4EE77FEA645C18BF7FEA655CD0
:100E500029D094EA050F08BF90EA020F05D054EAA2
:100E6000000C04BF1946104630BD91EA030F1EBFA7
:100E70000021002030BD5FEA545C05D140004941AB
:100E800028BF41F0004130BD14F580043CBF01F59E
:100E9000801130BD01F0004545F0FE4141F4700184
:100EA0004FF0000030BD7FEA645C1ABF194610465F
:100EB0007FEA655C1CBF0B46024650EA013406BF60
:100EC00052EA033591EA030F41F4002130BD00BF1F
:100ED00090F0000F04BF0021704730B54FF48064DC
:100EE00004F132044FF000054FF0000150E700BF5D
:100EF00090F0000F04BF0021704730B54FF48064BC
:100F000004F1320410F0004548BF40424FF00001A8
:100F10003EE700BF42004FEAE2014FEA31014FEAEB
:100F200002701FBF12F07F4393F07F4F81F060513A
:100F3000704792F0000F14BF93F07F4F704730B5A9
:100F40004FF4607401F0004521F0004120E700BF3C
:100F500050EA010208BF704730B54FF000050AE0C3
:100F600050EA010208BF704730B511F0004502D5C4
:100F7000404261EB41014FF4806404F132045FEAC6
:100F8000915C3FF4DCAE4FF003025FEADC0C18BF6B
:100F900003325FEADC0C18BF033202EBDC02C2F161
:100FA000200300FA03FC20FA02F001FA03FE40EAF3
:100FB0000E0021FA02F11444C1E600BF70B54FF0F3
:100FC000FF0C4CF4E06C1CEA11541DBF1CEA1355D5
:100FD00094EA0C0F95EA0C0F00F0DEF82C4481EA3D
:100FE000030621EA4C5123EA4C5350EA013518BF5D
:100FF00052EA033541F4801143F4801338D0A0FB4A
:1010000002CE4FF00005E1FB02E506F00042E0FBF6
:1010100003E54FF00006E1FB03569CF0000F18BFFC
:101020004EF0010EA4F1FF04B6F5007F64F54074A4
:1010300004D25FEA4E0E6D4146EB060642EAC62137
:1010400041EA55514FEAC52040EA5E504FEACE2EA4
:10105000B4F1FD0C88BFBCF5E06F1ED8BEF1004FA7
:1010600008BF5FEA500E50F1000041EB045170BD23
:1010700006F0004646EA010140EA020081EA030167
:10108000B4EB5C04C2BFD4EB0C0541EA045170BD63
:1010900041F480114FF0000E013C00F3AB8014F1DD
:1010A000360FDEBF002001F0004170BDC4F1000426
:1010B000203C35DA0C341BDC04F11404C4F12005A7
:1010C00000FA05F320FA04F001FA05F240EA020002
:1010D00001F0004221F0004110EBD37021FA04F638
:1010E00042EB06015EEA430E08BF20EAD37070BDF2
:1010F000C4F10C04C4F1200500FA04F320FA05F051
:1011000001FA04F240EA020001F0004110EBD37052
:1011100041F100015EEA430E08BF20EAD37070BDC2
:10112000C4F1200500FA05F24EEA020E20FA04F39B
:1011300001FA05F243EA020321FA04F001F000414A
:1011400021FA04F220EA020000EBD3705EEA430EBB
:1011500008BF20EAD37070BD94F0000F0FD101F0EA
:101160000046400041EB010111F4801F08BF013C23
:10117000F7D041EA060195F0000F18BF704703F061
:101180000046520043EB030313F4801F08BF013DE8
:10119000F7D043EA0603704794EA0C0F0CEA1355A4
:1011A00018BF95EA0C0F0CD050EA410618BF52EA5E
:1011B0004306D1D181EA030101F000414FF0000064
:1011C00070BD50EA410606BF1046194652EA430672
:1011D00019D094EA0C0F02D150EA013613D195EAE6
:1011E0000C0F05D152EA03361CBF104619460AD12E
:1011F00081EA030101F0004141F0FE4141F4700138
:101200004FF0000070BD41F0FE4141F4780170BD27
:1012100070B54FF0FF0C4CF4E06C1CEA11541DBF8C
:101220001CEA135594EA0C0F95EA0C0F00F0A7F88E
:10123000A4EB050481EA030E52EA03354FEA0131BB
:1012400000F088804FEA03334FF0805545EA1313CE
:1012500043EA12634FEA022245EA111545EA106596
:101260004FEA00260EF000419D4208BF964244F12D
:10127000FD0404F5407402D25B084FEA3202B61A4C
:1012800065EB03055B084FEA32024FF480104FF420
:10129000002CB6EB020E75EB030E22BFB61A754694
:1012A00040EA0C005B084FEA3202B6EB020E75EB27
:1012B000030E22BFB61A754640EA5C005B084FEA8F
:1012C0003202B6EB020E75EB030E22BFB61A75465C
:1012D00040EA9C005B084FEA3202B6EB020E75EB67
:1012E000030E22BFB61A754640EADC0055EA060E28
:1012F00018D04FEA051545EA16754FEA06164FEA6B
:10130000C30343EA52734FEAC2025FEA1C1CC0D116
:1013100011F4801F0BD141EA00014FF000004FF0A3
:10132000004CB6E711F4801F04BF01430020B4F164
:10133000FD0C88BFBCF5E06F3FF6AFAEB5EB030C1C
:1013400004BFB6EB020C5FEA500C50F1000041EB19
:10135000045170BD0EF0004E4EEA113114EB5C04E6
:10136000C2BFD4EB0C0541EA045170BD41F48011B9
:101370004FF0000E013C90E645EA060E8DE60CEAC1
:10138000135594EA0C0F08BF95EA0C0F3FF43BAFDE
:1013900094EA0C0F0AD150EA01347FF434AF95EA95
:1013A0000C0F7FF425AF104619462CE795EA0C0F79
:1013B00006D152EA03353FF4FDAE1046194622E746
:1013C00050EA410618BF52EA43067FF4C5AE50EA20
:1013D00041047FF40DAF52EA43057FF4EBAE12E710
:1013E0004FF0FF3C06E000BF4FF0010C02E000BFF1
:1013F0004FF0010C4DF804CD4FEA410C7FEA6C5CD4
:101400004FEA430C18BF7FEA6C5C1BD001B050EA76
:10141000410C0CBF52EA430C91EA030F02BF90EA61
:10142000020F0020704710F1000F91EA030F58BF20
:10143000994208BF90422CBFD8176FEAE37040F082
:10144000010070474FEA410C7FEA6C5C02D150EA20
:10145000013C07D14FEA430C7FEA6C5CD6D152EADB
:10146000033CD3D05DF8040B704700BF84461046A0
:1014700062468C461946634600E000BF01B5FFF79F
:10148000B7FF002848BF10F1000F01BD4DF808ED6F
:10149000FFF7F4FF0CBF012000205DF808FB00BF40
:1014A0004DF808EDFFF7EAFF34BF012000205DF89A
:1014B00008FB00BF4DF808EDFFF7E0FF94BF0120E7
:1014C00000205DF808FB00BF4DF808EDFFF7CEFFE8
:1014D00094BF012000205DF808FB00BF4DF808ED27
:1014E000FFF7C4FF34BF012000205DF808FB00BFF8
:1014F0004FEA410212F5001215D211D56FF478733C
:10150000B3EB625212D94FEAC12343F0004343EADE
:10151000505311F0004F23FA02F018BF40427047B9
:101520004FF00000704750EA013005D111F0004043
:1015300008BF6FF0004070474FF00000704700BFD9
:10154000FDF7BDFB002103E00A4B5B58435004311B
:1015500009480A4B42189A42F6D3094A02E000238E
:1015600013600432074B9A42F9D300F00DF880471C
:1015700070470000481D01000880FF1F6C85FF1F99
:101580000086FF1F24120020274C08B5F6F779FFCC
:10159000F6F7E0FFF7F746F9F7F758F9F7F762F8CB
:1015A000F7F72CFBFCF78EFBFCF776F9F7F7BDFCA1
:1015B000F7F7E8F9E08CF7F7E3FA2078F7F762F845
:1015C000E078F7F7CFF8F7F786FA28B1F7F783FA5C
:1015D0006070F7F780FAA060F7F7ECFA218960797C
:1015E000228AFCF7B3F9FDF7E3F8FDF781FA0F4B18
:1015F0004FF400725A60FAF743FCFBF723F90C4BE7
:1016000004225A60FAF76EFDFBF754F9FBF71BF959
:10161000F7F768FAF7F7A4FA0028F3D0FDF7C8F84F
:10162000FAF72EFCEEE700BF0C80FF1F80F00F40A2
:1016300000F00F4070B4860746D0541E002A41D0F7
:10164000CAB2034602E014F1FF343BD303F8012B86
:101650009D07F8D1032C2ED9CDB245EA05250F2CD4
:1016600045EA054519D903F110022646103E0F2E12
:1016700042F8105C42F80C5C42F8085C42F8045CEA
:1016800002F11002F2D8A4F1100222F00F0204F0CD
:101690000F041032032C13440DD91E462246043A7F
:1016A000032A46F8045BFAD8221F22F00302043210
:1016B000134404F003042CB1C9B21C4403F8011B09
:1016C0009C42FBD170BC704714460346C2E700BF82
:1016D0002DE9F84355EC104BC5F30A52A2F2FF3343
:1016E000132B064612DC002B41DB244A42FA03F39B
:1016F00005EA030252EA040017D105F0004302464E
:1017000086ED000B43EC102BBDE8F883332B1CDC7B
:10171000A2F213424FF0FF3323FA02F214EA020757
:101720001CD0A94624EA020803E04FF0000825EA8D
:10173000030942464B4620462946C6E90023FFF7E7
:1017400089FA41EC100BBDE8F883002205F0004354
:1017500086ED000B43EC102BBDE8F88305F0004349
:101760003A4686ED000B43EC102BBDE8F8830022CF
:1017700005F00043C6E90023BDE8F883FFFF0F0032
:10178000024B13B1024800F005B87047000000009A
:10179000A1170100002301461A46184600F01EB8A2
:1017A00038B50A4C0A4D641BA4100AD004F18043DA
:1017B000013B05EB8305013C55F804399847002CA3
:1017C000F9D1BDE8384000F0B3BA00BF481D0100B0
:1017D000441D0100704700BF704700BF2DE9F8436A
:1017E0002C4D0646286898460F469146FFF7F2FFB3
:1017F000294B1C68D4F84831002B3ED05A681F2A68
:101800001CDC02F1010E76B103EB82010124C1F868
:101810008890D3F8880194402043022EC3F88801B1
:10182000C1F8088123D00232C3F804E0286843F8E5
:101830002270FFF7D1FF0020BDE8F883174B0BB3F0
:101840004FF4C870AFF300800346D8B1D4F84821F4
:101850000260002141600A46C4F848014FF0010EC1
:10186000C0F88811C0F88C11002EDCD0CCE7D3F87A
:101870008C110C43C3F88C41D5E704F5A673C4F86A
:101880004831BBE72868FFF7A7FF4FF0FF30BDE8FE
:10189000F88300BF6885FF1F201D010000000000C5
:1018A00051EC100B2DE9F843C1F30A59A9F2FF35A9
:1018B000132D0C4610EE106A884610EE107A22DCCA
:1018C000002D52DB3E4B43FA05F901EA09030343BD
:1018D0001ED039A3D3E90023FFF7BEF9002200236D
:1018E000FFF7FCFD48B1002C04DD4FF4801343FAF0
:1018F00005F5A84428EA0904002723463A4643ECA4
:10190000102BBDE8F883332D06DDB5F5806F3FD091
:1019100041EC100BBDE8F883A9F213494FF0FF33F7
:1019200023FA09F910EA090FF2D023A3D3E900231F
:10193000FFF792F900220023FFF7D0FD0028DCD04A
:10194000002C09DD142D32D00127C5F1340507FA2A
:1019500005F5AE1928BFB844444626EA09072346D0
:101960003A4643EC102BBDE8F88313A3D3E90023D8
:10197000FFF772F900220023FFF7B0FD0028BCD06A
:10198000002C10DB54EA06070BD000270D4CB4E7FF
:1019900010EE102A0B46FFF75FF941EC100BBDE883
:1019A000F8833C46A9E700274FF00044A5E704F17F
:1019B0000108D1E7AFF300809C7500883CE4377ED6
:1019C000FFFF0F000000F03F51EC100BC1F30A5372
:1019D0002DE9F041A3F2FF35132D0C460F4610EE12
:1019E000106A1DDC002D43DB3D4B43FA05F801EA8C
:1019F0000803034319D038A3D3E90023FFF72CF9D8
:101A000000220023FFF76AFD20B1002C49DB27EA02
:101A1000080400262346324643EC102BBDE8F08133
:101A2000332D06DDB5F5806F32D041EC100BBDE8EB
:101A3000F081A3F213434FF0FF3828FA03F810EABD
:101A4000080FF2D024A3D3E90023FFF705F9002201
:101A50000023FFF743FD0028DCD0002C27DB3C46A9
:101A600026EA08062346324643EC102BBDE8F081F7
:101A700019A3D3E90023FFF7EFF800220023FFF7B3
:101A80002DFD0028C6D0002C1CDB00263446C1E703
:101A900010EE102A0B46FFF7DFF841EC100BBDE803
:101AA000F0814FF4801343FA05F52F44AFE7142D6E
:101AB00010D00123C5F1340503FA05F5AE1928BF8E
:101AC000FF18CCE724F00042064B324318BF1C46F7
:101AD00000269FE70137C2E79C7500883CE4377E0B
:101AE000FFFF0F000000F0BF80250000403800001D
:101AF000004B0000807000000096000000E1000034
:101B0000002C010000C201000084030090D00300FB
:101B100020A1070040420F0050C3000088130000BE
:101B2000018008080000000000000000C80000005C
:101B30000100C8000080000000000000000000005C
:101B40000000000000000000000000000000000095
:101B50000000000000000000010002000400080076
:101B60001000200001010100010000000000000041
:101B70000000000000010000000000000001000063
:101B80000000000001010100000000000000000052
:101B9000000100000000000001010100010100013E
:101BA0000100000001010100000000000000000031
:101BB000000100000000000001010100010100011E
:101BC0000100000000000000000000000000010112
:101BD0000100000100000000000000000000010101
:101BE000010000015780FF1F0400000009040000ED
:101BF000481C0100581C010000000000000000000B
:101C000000000000000000002E81FF1FEB80FF1F7E
:101C100000000000000000000000000000000000C4
:101C2000000000000000120043000000000000005F
:101C30000000000003010201100002020010000376
:101C400003011000000100005780FF1FB180FF1F3B
:101C50008B80FF1F6980FF1F043A2622B50901000F
:101C6000B1F2000049F30000B9F00000DD0401000A
:101C7000DD040100DD040100DD040100DD040100DC
:101C8000DD040100DD040100DD040100DD040100CC
:101C9000DD040100DD040100DD0401003BF600006D
:101CA000D1F5000031F60000FDF50000D1F500008F
:101CB000DD040100BDF50000A9F600007907010070
:101CC0004508010000000000450801000000000078
:101CD000390701006107010000000000A1060100B2
:101CE000D10601003909010019090100750601003A
:101CF00001010001010000000001010000000000DE
:101D000001010101010000000101000101000100C9
:101D10000001000001000036323130563130390008
:101D20004081FF1FF8B500BFF8BC08BC9E46704755
:0C1D3000F8B500BFF8BC08BC9E46704728
:081D3C0081170100358400004D
:041D44001184000006
:101D4800171D01000001020000080000010000004A
:101D58000200000000000000000000000000000079
:101D6800000000000000000000000000000000006B
:101D7800000000000000000000000000000000005B
:101D880000000000A1200000000002000000FF0485
:101D980003090400C2010000000800000000000060
:101DA8000022034200410044002000530054005226
:101DB8000049004E004700200049004E00440045FD
:101DC8000058002603530074006500700070006519
:101DD80000720020004D006F0074006F0072002038
:101DE8000044006500760020003A03540052004980
:101DF800004E0041004D004900430020004D006F97
:101E080000740069006F006E00200043006F006ED0
:101E180000740072006F006C002000200020002079
:101E280000200009024300020100C032090400003A
:101E3800010202000005240010010524010101042B
:101E480024020605240600010705830310000A0979
:101E5800040100020A0000000705810210000007C3
:101E680005020210000012010002020000103C2AC4
:101E78000001020001020001000000002C84FF1F85
:101E88009484FF1FFC84FF1F000000000000000076
:101E9800000000000000000000000000000000003A
:101EA800000000000000000000000000000000002A
:101EB800000000000000000000000000000000001A
:101EC800000000000000000000000000000000000A
:101ED80000000000000000000000000000000000FA
:101EE80000000000000000000000000000000000EA
:101EF80000000000000000000000000000000000DA
:101F080000000000000000000000000000000000C9
:101F180000000000000000000000000000000000B9
:101F280001000000000000000E33CDAB34126DE656
:101F3800ECDE05000B0000000000000000000000BF
:101F48000000000000000000000000000000000089
:101F58000000000000000000000000000000000079
:101F68000000000000000000000000000000000069
:101F78000000000000000000000000000000000059
:0422A8000012002000
:1022AC00481D01000880FF1F6405000000000000AD
:0822BC0000000000000000001A
:020000020000FC
:020000041FFFDC
:04800000000000007C
:040000031000154193
:00000001FF
